:1000000068C400009EC400009CC400009AC40000A4
:1000100098C4000096C4000094C4000092C400007C
:1000200090C400008EC400000C9419320C9401336B
:100030000C94CE3186C4000084C4000082C4000049
:1000400080C400007EC400007CC400007AC40000AC
:1000500078C400000C94F53174C4000072C4000030
:1000600070C400006EC400006CC400006AC40000CC
:1000700068C4000066C4000064C4000062C40000DC
:1000800060C400005EC400005CC400005AC40000EC
:1000900058C4000056C4000054C4000052C40000FC
:1000A00050C400004EC400004CC400000501090209
:1000B000A10185020901A1000509190129081500FE
:1000C0002501950875018102050109300931158165
:1000D000257F95027508810609381581257F9501D0
:1000E00075088106050C0A38021581257F95017572
:1000F000088106C0C005010980A101850319012AF4
:10010000B700150126B700950175108100C0050CD8
:100110000901A101850419012AA002150126A002E6
:10012000950175108100C005010906A1018506052C
:100130000719E029E71500250195087501810205D9
:1001400007190029EF1500250195F07501810205B9
:10015000081901290595057501910295017503910D
:1001600001C00660FF0961A1010962150026FF00B8
:100170009520750881020963150026FF00952075FA
:10018000089102C005010906A101050719E029E748
:1001900015002501950875018102950175088101F9
:1001A0000507190029FF150026FF0095067508812F
:1001B000000508190129051500250195057501910E
:1001C00002950175039101C00000000000000000CD
:1001D000000000000000000000000000000000001F
:1001E0000000000000000000000000007E0F00D4AE
:1001F000FFFFFFC7000000780000000000000000C3
:100200002A2B280000000000000000000000000071
:1002100000000029000000002C1E3420212224347C
:100220002627252E362D3738271E1F20212223244E
:1002300025263333362E37381F0405060708090AEA
:100240000B0C0D0E0F101112131415161718191A86
:100250001B1C1D2F3130232D350405060708090A04
:100260000B0C0D0E0F101112131415161718191A66
:100270001B1C1D2F3130354C09025B00030100A00F
:10028000FA09040000010301010009211101000124
:10029000224400070581030800010904010002034C
:1002A000000000092111010001222200070582033C
:1002B00020000107050303200001090402000103D7
:1002C00000000009211101000122B6000705840386
:1002D0002000011201000200000008EDFE000001F4
:1002E00000010203011C037600690061006C003A02
:1002F00000660036003400630032006200330063A1
:100300000000000C036D00620074006B006C0000C4
:100310000014036D0065006C006F006E00620072D7
:1003200000650064000000040309043A003B003C3F
:10033000003D003E003F00400041004200430044B9
:100340000045004C004A004B00290014001A000828
:1003500000150017001C0018000C00120013002AE2
:1003600000460049004E002B21040016000700093A
:10037000000A000B000D000E000F003300280000E3
:100380000000000000E1001D001B00060019000530
:100390000011001000360037003800E50000005260
:1003A00000000022520000E20000002C410000008A
:1003B000002C000000E6000000E700500051004F54
:1003C000003A003B003C003D003E003F0040004141
:1003D0000042004300440045004C004A004B0035F9
:1003E000003400010052000100010001000100245E
:1003F00000250026004C000000000000003900012C
:1004000000500051004F000100540056002100220E
:100410000023002800000000000000E1002D002E55
:10042000002F0030003100550057001E001F002033
:1004300000E50000000000000001000100000000D5
:1004400000010000000000000000000000000000AB
:10045000000000000000000000000000000000009C
:10046000000000000000000000000000000000008C
:10047000000000000000000000000000000000007C
:100480000000000000000000000000A900000000C3
:10049000000000000000000000000000000000005C
:1004A000000000000000000000000000000000004C
:1004B000000000000000000000000000000000003C
:1004C00000E600E4004C00AA00000000000000006C
:1004D000000000000000000000000000000000001C
:1004E00000000000000000000000000000222325A2
:1004F0002628292A2C2D2F3032333536383A3B3DE9
:100500003E4042434547494A4C4E50515355575936
:100510005A5C5E6062646668696B6D6F7173757753
:10052000797B7D7F81838587898A8C8E9092949652
:10053000989A9C9E9FA1A3A5A7A8AAACAEAFB1B361
:10054000B4B6B8B9BBBCBEBFC1C2C3C5C6C7C9CAB1
:10055000CBCCCDCED0D1D2D2D3D4D5D6D7D7D8D973
:10056000D9DADADBDBDBDCDCDCDCDCDDDDDDDDDCD1
:10057000DCDCDCDCDBDBDBDADAD9D9D8D7D7D6D5E3
:10058000D4D3D2D2D1D0CECDCCCBCAC9C7C6C5C3A5
:10059000C2C1BFBEBCBBB9B8B6B4B3B1AFAEACAAF2
:1005A000A8A7A5A3A19F9E9C9A98969492908E8CA2
:1005B0008A89878583817F7D7B79777573716F6D7C
:1005C0006B6968666462605E5C5A59575553515056
:1005D0004E4C4A4947454342403E3D3B3A3836350A
:1005E0003332302F2D2C2A292826252322FFAA7FBB
:1005F0005540000101010101010101010202020255
:1006000002020202020303030303030303040404BC
:100610000404040405050505050606060606070785
:1006200007070708080808090909090A0A0A0B0B3D
:100630000B0C0C0C0D0D0D0E0E0E0F0F0F101011DC
:100640001111121213131414151516161717181862
:1006500019191A1A1B1B1C1D1D1E1E1F20202122CA
:1006600022232424252626272829292A2B2C2D2D10
:100670002E2F30313232333435363738393A3B3C2D
:100680003D3E3F404142434445464748494A4C4D20
:100690004E4F50515354555658595A5B5D5E5F61E9
:1006A0006264656668696B6C6D6F7072737577787C
:1006B0007A7B7D7E8082838587888A8C8E8F9193DA
:1006C0009596989A9C9EA0A2A3A5A7A9ABADAFB101
:1006D000B3B5B7BABCBEC0C2C4C6C9CBCDCFD1D4E6
:1006E000D6D8DBDDDFE2E4E7E9EBEEF0F3F5F8FA8C
:1006F000FDFF1E0F057F3F1F643214643214783CE7
:100700001E1E140A05FD377A585A000004E6D6B4B6
:10071000460200210116000000742FE5A3E0043812
:10072000018C5D003D8889C65436C3174FE4F60638
:100730004D5663408D2D851E4D36EBDAC892A1547F
:100740006CFF9AB9D52D84C03F9973B2EA4EA8AD1B
:1007500085308452CE8640435E2222914DD6F3737B
:10076000F2BEA0E103EACDE402338970AED3B00C4F
:10077000F277EFC527F580D3EAC4CF0087B18E5654
:100780001AEC3059EE23870222B04DC4FACEFA3E5D
:1007900044BC7BFFA837D7F4EAD3173E80050CA8EA
:1007A0009B01DFDB3E352375A8A45814B9B5209B07
:1007B0001EEC8B6F390819D9B7FB304B00AD4BAB32
:1007C000B8A2CF8AF06EB4DEBDE5FC3888DCA001AB
:1007D0003CC8DC05AA77616231D5EF67B8787D4AFD
:1007E000A4CFF75784FB7A2315234B7B0D22C76ACE
:1007F0007D9C2FC28B4446BDC24B5261D633E69DD1
:100800004386912AE919DA6C7F2098B0FEE621CD63
:100810006AE068A0340268776C81E06C6AA6B8551B
:1008200031543D26D21A90597DFE2E84F3F1F35BAC
:10083000C5CEB75E58252903D55A7DA93A0E87AB98
:10084000906F9741451C8774263EF96F6B727A1D35
:1008500087B59532866ABBE0FC8690A53A35C63EE0
:10086000C6B1818E52A6FEC9D85B1989E6AFCC58B5
:100870006B852A05A7303169AB9A7A53E6EFEF7999
:10088000294DF88636CD5350C4E670F5E0F6A764DE
:10089000B84074C3EE031A73471AAB8183C2C871A0
:1008A0006B651519E5DADA2539CE0AB95B9E3F5B2F
:1008B000003FBBBC04F249040B0001A803B90800C7
:1008C00000266DD31FB1C467FB020000000004596D
:1008D0005A0011241FBECFEFDAE0DEBFCDBF04B651
:1008E00003FE18C08091730590917405A091750561
:1008F000B09176058730904BA740B04B59F41092D9
:100900007305109274051092750510927605E0E05B
:10091000F8E3099525E0A4EEB1E001C01D92A337EC
:10092000B207E1F711E0A0E0B1E0EEE9FBE602C0BA
:1009300005900D92A43EB107D9F70E94CB290C94E3
:1009400048355ECB9C019A9581159F4118F5F32F90
:10095000F270EE27832F8170732F74706627532FE8
:100960005870442734FF0CC08295807FEF2B09F02C
:100970008062672B09F08064452B69F080680895D8
:10098000EF2B09F08260672B09F08460452B19F08A
:100990008860089580E00895CF93DF93EB01D2DF64
:1009A000FE010995DF91CF91089580936F05089519
:1009B00080937005089521E030E001C0220F8A95F0
:1009C000EAF780917005822BF3CF21E030E0A90196
:1009D00002C0440F551F8A95E2F7CA018095909195
:1009E00070058923E5CF292F953090F58F3080F55C
:1009F00090E03FE0239F800D911D1124282F277048
:100A000041E001C0440F2A95EAF723E096958795C7
:100A10002A95E1F7FC01EE0FFF1FE80FF91FEF58D1
:100A2000FC4F20E030E070E05191DF01CB01022E5D
:100A300002C0969587950A94E2F781708195852783
:100A4000842385278E932F5F3F4F2330310561F735
:100A50000895292F953078F58F3068F590E03FE0C4
:100A6000239F800D911D1124682F677023E09695B8
:100A700087952A95E1F7FC01EE0FFF1FE80FF91F9C
:100A8000EF58FC4F40E050E080E0219130E0062E2E
:100A900002C0369527950A94E2F721703327042E79
:100AA00001C0220F0A94EAF7822B4F5F5F4F433059
:100AB000510559F7089580E008959091700521E05F
:100AC00030E0F90101C0EE0F8A95EAF7D90102C0C2
:100AD000AA0FBB1F6A95E2F7EA2B01C0220F4A95C5
:100AE000EAF7892F8E23E81303C0892F822B60CF6A
:100AF0002095822F8923FBCF80911F0390911E03A5
:100B0000981301C008958F5F8770FACF9091BB044E
:100B1000809589238093BB04282F2770211110C052
:100B2000891771F09091720592FF0AC0869586959B
:100B300086954BDF1092BB041092BD041092BC044A
:100B40000895982F90958091B80489238093B804D4
:100B500008958091B704811531F01092B704109276
:100B6000BF041092BE040895803E9105D9F1C8F4E7
:100B70008133910509F482C048F48932910509F462
:100B800072C08A32910509F480C0089589339105B5
:100B9000E9F082389105D1F08533910509F45EC002
:100BA0000895843E9105D9F148F4823E910539F1CA
:100BB000833E910549F181EE90E00895863E9105CE
:100BC000C9F1873E910509F43EC008952091710551
:100BD0002370211164C02091720523FF14C089E2A3
:100BE00090E008952091710520FD45C03091720577
:100BF00030FF09C024FD24C083EE90E008952091C9
:100C0000710522FDF7CF08952091710522FD44C0A2
:100C10003091720530FD43C024FFF5CF11C0209103
:100C2000720521FFF0CF8091710584FD09C087EE28
:100C300090E008952091710523FFE5CF24FFF7CFC1
:100C400080E090E008952091710523FD2BC0309144
:100C5000720531FFE1CF84EE90E008952091710597
:100C600025FFD1CFBCCF2091710525FD1EC020915D
:100C7000720523FFC8CF89E390E0089520917105A4
:100C800026FFC1CF8AE290E008952091710526FFEA
:100C9000BACF81E390E0089582EE90E0089580EE6F
:100CA00090E0089586EE90E0089585E390E0089541
:100CB0009091710592FF10C041E0282F24712430DB
:100CC00009F040E031E0282F2871283009F030E0A9
:100CD000431711F02CE0822793FF10C041E0282F2A
:100CE0002471243109F040E031E0282F28712831A7
:100CF00009F030E0431711F02CE0822730917205A3
:100D000030FF10C051E0282F2171213009F050E050
:100D100041E0282F2871283009F040E0541711F0E5
:100D200029E0822731FF10C041E0282F21712131B5
:100D300009F040E031E0282F2871283109F030E037
:100D4000431711F029E0822794FD877E08951F93B1
:100D5000CF93DF9309DFEC01811522E5920708F0BC
:100D600052C0811540E5940708F0CDC0803E910542
:100D700020F58D3C910508F0A1C0883A910570F4EA
:100D8000853A910508F097C081309105B9F1049733
:100D9000813A910598F1C0E0D0E030C0885A9109BD
:100DA0004B97C8F7C85AD0E0CC0FDD1FC858DE4FAC
:100DB0000990D881C02DD46421C0811550E49507D5
:100DC000B0F4C11580E2D80708F0B3C0C83ED10521
:100DD000A8F0CE019A9581159F41E8F68D2F68DF26
:100DE000182FCE019927C0DEEC01D12B07C099271F
:100DF000BBDECC27DF70C82BD92BD06ACE01DF91A8
:100E0000CF911F910895803842E59407C8F5803648
:100E100052E5950708F05BC0C03482E5D807D0F4EE
:100E2000C03292E5D90708F04BC08C2F8695869585
:100E300020E2829FC0011124C37021E030E0A901AB
:100E400002C0440F551FCA95E2F7EA01C82BD92BFF
:100E5000DD68D4CF8C2F86958695877050E2859F6C
:100E6000C0011124C37021E030E0A90102C0440F89
:100E7000551FCA95E2F7EA01C82BD92BDC68BECF13
:100E8000803C52E5950758F48F71C03AD245A0F5E1
:100E900090E0982F8827EC01C46FD06AAFCF805CB8
:100EA0009245809708F077CFDC2FCC27CC27DF71D5
:100EB000C06FD06AA3CFA497D064A0CFD0659ECFD7
:100EC000CF71D0E0DC2FCC27C16FD06A97CF869549
:100ED0008695877020E2829FC0011124C37021E0B3
:100EE00030E0A90102C0440F551FCA95E2F7EA019C
:100EF000C82BD92BDA6882CFDBDEC82FD0E0DC2FFD
:100F0000CC27D0627BCF8F71D3DE93E0CC0FDD1F77
:100F10009A95E1F7CC27DF70282F30E084FF05C0D9
:100F200050E1859F900111243327C22BD32BD06928
:100F300065CF8D2F8F71BCDE182FCE01992714DE5F
:100F4000EC01D12BDECF80E00895F894E82FE295F4
:100F5000EF70F0E041A18F7021E030E0B90102C0F4
:100F6000660F771F8A95E2F7CB01962F9095942311
:100F700091A392A1892B82A3789408950895CF928A
:100F8000DF92EF92FF921F93CF93DF93172FE82FFB
:100F9000F0E0EE50FA4F71110CC0E4918E2F7E2FCD
:100FA0006E2FDF91CF911F91FF90EF90DF90CF9048
:100FB0000895E62EF12CC72ED12CF491EF2F86E068
:100FC000689F90011124CFEFD0E0C901BE010E94BB
:100FD0006533AB01EE0CFF1C65E5649FC001659FA6
:100FE000900D1124E81AF90A6E2D660F6E0D7E0120
:100FF000EC18FD08FE9DD001FF9DB00D11248B2F34
:10100000169F70011124EF2CFF246E01CE18DF080B
:101010007601FE9D6001FF9DD00C11247E01E61A31
:10102000F108B701169F7001179FF00C1124EF2CE7
:10103000FF24CE19DF09FC9F7001FD9FF00C1124E5
:101040007F2D43305105C1F02C3F334058F44130DF
:101050005105B1F04230510509F0A2CFEB2F8F2D91
:101060007F2F9ECF4430510571F04630510509F471
:1010700097CF7B2F8D2D94CF7D2DEB2F8F2F90CF62
:101080007F2FED2D8DCFEF2D7B2FF8CFCF93982F86
:10109000762F842FC22F692F72DF472F282F8C2F96
:1010A00090E090D1CF9108958091AF04843028F4DE
:1010B000837084608093AF040895843AE8F383706A
:1010C000806AF8CFCF93DF938091AF0480FD0BC08F
:1010D000C0E0D0E020E040E060E0CE0173D1219696
:1010E000C530D105B9F714D6DF91CF910895FF929D
:1010F0000F931F93CF93DF93182F062FF42E809119
:10110000AF0480FF0CC0C0E0D0E02F2D402F612F36
:10111000CE0158D12196C530D105B9F7D3DFCDB76F
:10112000DEB7E5E00C94C233982F762F842F209100
:10113000AF0420FF07C0692F22DF962F672F482FAB
:10114000892FD5CF0895CF93DF93EC01EFEAF4E038
:10115000438162818C81E8DF8C818F5F8C83DF919A
:10116000CF910895CF93DF93EC01EC81F0E0E35150
:10117000FB4F4491EFEAF4E062818181D5DF8C81FD
:101180008F5F8C83DF91CF910895FF920F931F9310
:10119000CF93DF93EC01F12C00E010E08C819801FB
:1011A0004091B2046091B1048F0D70DF0F5F1F4F4B
:1011B00083E3F80E0530110589F784DF8C819A816D
:1011C00090FF07C08F5F8C83CDB7DEB7E5E00C944E
:1011D000C2338150F8CFEF92FF920F931F93CF93BA
:1011E000DF93FC018281FF24F39480FF02C0FF247F
:1011F000FA94C0E0D0E020E040E060E0CE01E2D030
:1012000004E010E0E12C8091B1028E0D86308CF16B
:1012100065E00E945833892F082E001C00088C17A7
:101220000D0679F44091B2040403A00111245595F0
:101230004795559547959E016091B1048091B00402
:1012400025DFEF0C01501040F1F62196C530D10595
:1012500091F638DF8091B102F1E0FF120EC08115E6
:1012600091F081508093B102CDB7DEB7E6E00C94E7
:10127000C13387FFD1CF8B5FCFCF90E00196BE0106
:101280000E947933EFCF84E0EDCFCF93DF93C0E0BE
:10129000D0E020E040E060E0CE0194D02196C5305F
:1012A000D105B9F7C0E0D0E08091B002082E001C53
:1012B0000008C817D0055CF180910501082E001CBC
:1012C00000088C170D061CF19E014091B20460913C
:1012D000B1048091B004DADE2196C530D10521F742
:1012E000F1DE809104019091B002980F9093B002CA
:1012F00020910501280F20930501121614F4943053
:101300001CF0819580930401DF91CF91089520E036
:1013100040E060E0CE0156D0DFCF0F931F93CF9314
:10132000DF93EC0120E030E06091B1048091B004E3
:101330009C8189010F5F1F4F223031053CF49115CC
:1013400041F04091B204A2DE9801EECF4091B20488
:10135000911140E09BDE98010530110529F7B2DEBE
:101360008C8190E00196817099278C83DF91CF91D9
:101370001F910F91089581152CE7920741F4209158
:10138000EB023091EC02232B11F480E090E0089501
:10139000E7E2F4E080E090E067E977E24AEB57E2C9
:1013A0002CE238E277836683518740873387228730
:1013B00097878687019670968830910599F70895EA
:1013C000509A0895FC01EE0FFF1FE80FF91FE15D31
:1013D000FD4F61834083228308951092010510928E
:1013E0000005E0ECF4E08581811102C014821682D0
:1013F000379684E0E83FF807B1F70895AC013091E3
:10140000030560910205232F621301C00895822F06
:1014100090E0FC01EE0FFF1FE850FB4F0190F081C0
:10142000E02DE417F50791F467E0649FF001659FF4
:10143000F00D1124E054FB4F41E044832313E6CF29
:101440000196837099278093030508950196282FAC
:101450002370DACFFC018481862381110AC0828146
:101460008115B9F06823908593FF05C081E0611173
:101470000FC080E00895282F22952F708F70282BA1
:10148000962F92959F706F70962B81E02913F1CF64
:10149000089581E00895282F35EB2303C00111241E
:1014A00097FF04C080589109892F089580589F4F55
:1014B000FBCF8091910380FD14C081FD14C082FD9B
:1014C00016C080919003811581F08E3180F420E563
:1014D000829FC00111246EE170E00E947933862F53
:1014E000089584E1089588E2089588E0089580E5EC
:1014F00008958091910380FD17C081FD17C082FD82
:1015000019C080918F03811599F0883298F428E0F2
:10151000829FC001112468E270E00E947933611556
:10152000710551F0862F089562E0FCCF64E0FACF98
:1015300061E0F8CF68E0F6CF81E00895FA013097D6
:1015400009F009950895E0911403F091150330977F
:1015500039F00190F081E02D309711F00995089550
:1015600080E00895A3E0B0E0E8EBFAE00C94A93342
:101570009C0180912C0290912D0282179307B1F06B
:1015800030932D0220932C02E0911403F091150367
:10159000309761F00084F185E02D309739F083E0D9
:1015A00089833B832A83CE01019609952396E2E045
:1015B0000C94C533A3E0B0E0E0EEFAE00C94A9335C
:1015C0009C0180912A0290912B0282179307B1F01F
:1015D00030932B0220932A02E0911403F09115031B
:1015E000309761F00084F185E02D309739F084E088
:1015F00089833B832A83CE01019609952396E2E0F5
:101600000C94C53390911F01913091F0A8EEB1E098
:10161000EFEF90E02D91821751F0EF3F19F4211177
:1016200001C0E92F9F5F9630A9F7EF3FC9F40895F5
:101630009091710597FFEACFE82FE695E695E6953C
:10164000803FA8F7F0E0E251FE4F877021E030E0E4
:1016500001C0220F8A95EAF78281822B8283089546
:101660000E2E000CFF0BEA51FE4FF8CF90911F0198
:10167000913021F49091710597FD0CC0E8EEF1E0F6
:101680009191891302C0DF011E9251E0EE3EF507F1
:10169000B9F70895E82FE695E695E695803FC8F7F7
:1016A000F0E0E251FE4F877021E030E0A90102C076
:1016B000440F551F8A95E2F7CA01809592818923CC
:1016C0008283089580911E0108952FB7F894809128
:1016D000260290912702A0912802B09129022FBFE3
:1016E0000895CF93DF93C091B8048091BA04C82BBA
:1016F0008091B7048115F1F0E8DF2091BE043091AC
:10170000BF04821B930B8838934108F022DAD091F2
:10171000B70480911F01813021F48091710587FD0C
:1017200013C086E028EE31E090E0815088F49111FA
:1017300010DACD2B8091A30380958C239091A20386
:10174000892BDF91CF9108958EE120EF31E0ECCF2E
:10175000F90141919F01411541F39F5FE6CF962F1B
:101760002091720522FF0EC0682F660F660F660F6C
:10177000692B6093BB041FD9A8DF9093BD048093AD
:10178000BC04089518C99091B704292F2823211566
:1017900059F0809589238093B704811531F095DF46
:1017A0008093BE049093BF04089580E090E0F8CF4A
:1017B0008CDF2091940330919503232B211521F088
:1017C0008093DA029093DB02209196033091970385
:1017D000232B211521F08093D8029093D902E09118
:1017E0001403F0911503309759F00680F781E02D2E
:1017F000309731F082E08093920382E993E009957B
:101800000895611509F441C0E3E3E80FE33148F4BA
:10181000F0E0E65BFA4C0C948C334BDE81958093C0
:101820009503C6CF46DEFBCF44DE819580939403BB
:10183000F8CF3FDEFBCF5DDE80939603F2CF59DE1B
:101840008195FACF56DE819580939703EACF51DEDA
:10185000FBCF815D990B21E030E001C0220F8A951A
:10186000EAF780919303822B80939303DACF8091E0
:101870009103816080939103D4CF80919103826022
:10188000F9CF809191038460F5CF409194038D3C12
:1018900059F48091950387FF0DC01092950341156F
:1018A00059F41092900308C08E3C81F48091950306
:1018B00018169CF3411581F080919603909197033F
:1018C000892B8111AECF10928F03ABCF8F3C41F4A7
:1018D00047FFF0CF10929403809195038115E0CFDC
:1018E000803D19F41416B4F3E5CF90919603893D29
:1018F00029F41916FCF610929603DCCF8A3D19F4F0
:1019000097FFD8CFF8CF909197038B3D29F497FF9D
:10191000D1CF10929703CECF8C3D19F41916CCF38A
:10192000C9CF9FE2980F983090F4815D990B21E028
:1019300030E0B90102C0660F771F8A95E2F7CB014C
:10194000809590919303892380939303B3CF8D3D2A
:1019500031F4809191038E7F80939103ABCF8E3DC4
:1019600021F4809191038D7FF7CF8F3D09F0A2CFB5
:10197000809191038B7FF0CF2FB7F894609126026E
:101980007091270280912802909129022FBF08951B
:10199000CF92DF92EF92FF92CF93DF93D82FC92F90
:1019A000C0902104D0902204E0902304F0902404FD
:1019B000E3DF6C197D098E099F09643F7140810541
:1019C000910510F1D9DF6B017C0182E390E0A0E08A
:1019D000B0E0C092CE02D092CF02E092D002F0925C
:1019E000D1028093CA029093CB02A093CC02B09311
:1019F000CD02D0931F04C0932004DF91CF91FF90BC
:101A0000EF90DF90CF90089584EF91E0A0E0B0E0F8
:101A1000E0CFFC019B0180911C0290911D02861772
:101A2000970740F0672B29F48091E8008E77809328
:101A3000E800C90140E0009741F4411106C08091DF
:101A4000E80082FF2FC080E008952091ED0221156B
:101A5000A9F12530A9F12091E80023FD2DC02091A6
:101A6000E80022FDECCF2091E80020FFE4CF309188
:101A7000F3002091F200009719F02830310558F05A
:101A800041E02830310509F040E02091E8002E7750
:101A90002093E800D0CF41914093F10001972F5F50
:101AA0003F4FE9CF8091ED02811541F0853041F043
:101AB0008091E80083FFC3CF81E0089582E008951C
:101AC00083E008958091160287FF13C08091E8009B
:101AD00082FF06C08091E8008B778093E80008952C
:101AE0008091ED028111F2CF08958091ED02811570
:101AF000D9F38091E80080FFF8CF8091E8008E77DD
:101B0000ECCF2091E4003091E50095E6A901209109
:101B1000EC00822F817020FF06C08091E80080FFDA
:101B200006C080E008952091E80022FD1AC080914F
:101B3000ED02811589F0853089F08091EB0085FDFB
:101B40000FC02091E4003091E50042175307F9F2ED
:101B50009A95E1F684E0089582E0089583E008957F
:101B600081E00895E8EDF0E080818E7F808310921F
:101B7000E2001092DA001092E100A0EEB0E08C9149
:101B800081608C9380818F77808319BCA7EDB0E052
:101B90008C918E7F8C9380818F7E80831092150232
:101BA0000895E0911403F0911503309739F0028401
:101BB000F385E02D309711F060E209950895982F94
:101BC0009093E900891771F07091EC002091ED007D
:101BD0005091F00021FD09C09F5F973089F78093F5
:101BE000E9000895762F242F50E03091EB003E7FDE
:101BF0003093EB003091ED003D7F3093ED0030915C
:101C0000EB0031603093EB007093EC002093ED001B
:101C10005093F0002091EE0027FDDECF0895A0E064
:101C2000B0E0E5E1FEE00C94A333C8EDD0E088819C
:101C30008F7E8883E7EDF0E080818160808384E09F
:101C400082BF81E08093150288818E7F888302EEB7
:101C500010E0F80110821092DA0081EEC82ED12C2B
:101C6000F601108288818F778883888180688883D5
:101C700088818F7D888319BC1092ED021092140226
:101C80001092BE021092130290EEE92EF12CF70191
:101C900080818B7F808388818160888342E060E0DF
:101CA00080E08DDFF60180818E7F8083F801808166
:101CB00081608083808188608083F70180818E7F4E
:101CC0008083888180618883CDB7DEB7E8E00C949B
:101CD000BF33E0911F0390911E0329E0E91302C076
:101CE00080E00895AE2FB0E02E9FF0011124E05E59
:101CF000FC4F3181361306C03081381303C0358163
:101D0000341304C0FD013196E770E8CF81E00895F7
:101D10003BB13E7F2BB121604FB7F8948FE292E048
:101D2000FC010196508168E02BB9000000C057FF0C
:101D30003BB9550F000000C000C000C03BB900C057
:101D40006A9591F752E08E33950751F74FBF8FE5B3
:101D500094E00197F1F700C00000089581E08093BE
:101D6000E00080E28093D8001092C9008FE19EE4E9
:101D70000197F1F700C0000087E090EBDC01809351
:101D8000730590937405A0937505B093760588E16B
:101D90009CE00FB6F894A895809360000FBE9093D6
:101DA0006000FFCF0F931F93CF93DF938B01EA0166
:101DB0009091ED02943051F58093E9008FEF90916E
:101DC000E80095FD06C095ED9A95F1F700008A951B
:101DD000B1F78091E80085FF19C093DE811111C031
:101DE0008091E80085FD06C08091E8008E778093A1
:101DF000E800F3CFF80181918F018093F1002197E2
:101E000079F78091E8008E778093E800DF91CF9199
:101E10001F910F910895792F603229F440E250E02C
:101E2000682F82E0BFCF0895CF93DF93D82FC92FBB
:101E300048E050E0682F792F81E0B4DF88E0ED2F93
:101E4000FC2FAEE1B2E001900D928A95E1F7DF91AF
:101E5000CF910895BC0140E250E084E0A3CFBC01E3
:101E600046E050E084E09ECFBC0143E050E084E0D7
:101E700099CF9091720592FB222720F9281779F0CB
:101E800080FB92F9909372056091710570917205D3
:101E900084E090E00E94D03482E00C94860508959E
:101EA0001F93CF93DF93962F122F632F8430D8F494
:101EB0009530C8F44F30B8F4C42FD0E0CC0FDD1FFC
:101EC0002EE1929FC00DD11D112496E9899FC00D6E
:101ED000D11D1124CE0189960E94B634612FCE0106
:101EE0008A960E94B634DF91CF911F910895809118
:101EF0001F01813061F58091710587FF28C0F1DBFA
:101F00008093EF0140E250E064EF72E08EEE91E0EA
:101F10000E947134892BD1F080E2EEEEF1E0A4EF63
:101F2000B2E001900D928A95E1F7E0911403F091EF
:101F30001503309759F00480F581E02D309731F08A
:101F400086E08093EE018EEE91E009950895C9DB5D
:101F50008093E60148E050E066E173E086EE91E0B0
:101F60000E947134892B91F388E0E6EEF1E0A6E15E
:101F7000B3E001900D928A95E1F7E0911403F0919E
:101F80001503309719F30280F381E02D3097F1F2B9
:101F900086EE91E0DACF811531F09091B804892B6B
:101FA0008093B804A4CF0895811531F09091BA04BC
:101FB000892B8093BA049BCF0895CF93C82F8115A6
:101FC000C1F08CEF8C0F813A80F580911F01813038
:101FD00021F48091710587FD0EC0E8EEF1E081915A
:101FE000C817F9F021E0EE3EF207C9F78C2F0ADBA3
:101FF0007EDFCF910895EC2FE695E695E695F0E02B
:10200000E251FE4F828190E04C2F477021E030E09A
:1020100002C0220F331F4A95E2F782239323892BB4
:1020200029F38C2F23DB63DFE1CF80E28C0F883034
:1020300068F4C77081E090E001C0880FCA95EAF7A4
:10204000C091B804C82BC093B804D2CF8BE58C0FD5
:10205000833030F42C2F2452330BC90183DAC9CFDB
:10206000E8E5EC0FEB3148F4F0E0EE0FFF1FE2552E
:10207000FE4F808191819EDABCCF83E38C0F833148
:1020800008F0B7CF61E08C2FBCDBB3CFCF93DF93E9
:10209000EC01805E9109089720F064ED7FE02097C5
:1020A00011F46BEC7FE0CE010E94CC048C2F85DF15
:1020B000DF91CF910895811541F19CEF980F913AEE
:1020C00010F4D4DA14CF90E2980F983050F487705F
:1020D00091E001C0990F8A95EAF7892F0E94A10526
:1020E000F1CF9BE5980F933018F480E090E03ACA66
:1020F00098E5980F9B3118F480E090E05BCA93E379
:10210000980F933110F460E07CCB08951F93CF9328
:10211000DF93182FEB0151DF209731F4812FCBDFB4
:10212000DF91CF911F9108958FE99FE00197F1F71B
:1021300000C000002197F0CF811519F00E94A10581
:10214000D6CE0895811539F080959091BA048923EF
:102150008093BA04CCCE08951092B80480911F01E8
:10216000813011F58091710587FF1EC0E0EFF1E02D
:102170008EE1DF011D928A95E9F780E090E0F2D9C7
:1021800080E090E017DA1092BA04B1DE86E0E2E96E
:10219000F3E0DF011D928A95E9F710929003109207
:1021A0008F031092910304CBE8EEF1E086E0E1CFDB
:1021B000D3DF2FEF84E39CE0215080409040E1F793
:1021C00000C0000088E19CE00FB6F894A8958093C9
:1021D00060000FBE90936000FFCFAAE2B0E0E3EF93
:1021E000F0E10C94A83386E192E0FC010196209185
:1021F000F100208322E08E319207B9F78091170217
:10220000893009F457C0C8F4823009F4B2C0833071
:1022100009F482C0813081F18091E80083FFE6C03B
:1022200080911602909117029A3008F0DFC0E92FD2
:10223000F0E0E35AFA4C0C948C338A3009F489C0EC
:102240008B3051F780911602813231F780911A025A
:1022500090911B02892B01F78091E800877F809382
:10226000E80030DC81E090911802911101C080E01B
:1022700080931F0171DFD0CF80911602813A61F601
:102280008091E800877F8093E80080911A02909106
:102290001B02892B59F060E080E090E070E0B9DB30
:1022A0008091E8008B778093E800B6CF68E08EE1FC
:1022B00092E0F4CF80911602813209F0ADCF809187
:1022C0001A0290911B028D7F892B09F0A5CF809176
:1022D000E800877F8093E8008091E80082FF17C0C4
:1022E0009091F3008091F200029731F48091F10017
:1022F000813011F0863021F48091F10080931E012D
:102300008091E8008B778093E800DCDB85CF8091BB
:10231000ED028111E1CF80CF80911602813A09F060
:102320007BCF80911A0290911B02892B09F074CF08
:102330008091E800877F8093E8008091E80080FF2B
:10234000FCCF80911F018093F1008091E8008E778F
:10235000DACF80911602813209F05ECF8091E800D9
:10236000877F8093E800AEDB8091190280931D0186
:1023700053CF80911602813A09F04ECF8091E80048
:10238000877F8093E8008091E80080FFFCCF8091F8
:102390001D01D9CF803889F0823841F580911A0229
:1023A0008F70873018F58093E9008091EB0085FBF2
:1023B000882780F91092E90006C08091BE02880F3C
:1023C00090911302892B9091E800977F9093E800F9
:1023D0008093F1001092F1008091E8008E7723C085
:1023E000811116C080911802813009F18091E800B6
:1023F00083FF0AC08091E800877F8093E800809186
:10240000EB0080628093EB00AA96E3E00C94C43367
:10241000823061F780911802811581F01092E900F5
:102420008091E800877F8093E8004CDBDFCF81E07C
:10243000933009F080E08093BE02F0CF80911A02C1
:102440008F702FEF280F263088F68093E9002091B7
:10245000EB0020FFE3CF933031F48091EB008062FA
:102460008093EB00DBCF9091EB0090619093EB00B9
:1024700021E030E0A90102C0440F551F8A95E2F720
:102480004093EA001092EA008091EB008860E8CF68
:102490008111ACCF109118021F778091E3008078F2
:1024A000812B8093E3008091E800877F8093E80090
:1024B00009DB8091E80080FFFCCF8091E300806819
:1024C0008093E30083E0111101C082E08093ED026C
:1024D0008DCF8058823008F089CF8091180290917A
:1024E00019028C3D53E0950791F583E08A838AE2D7
:1024F00089834FB7F894DE01139620E03EE051E265
:10250000E32FF0E050935700849120FF03C08295A1
:102510008F703F5F8F708A30C0F0895C90E08D9340
:102520009D932F5F243161F74FBF8091E800877F33
:102530008093E8006AE270E0CE0101966ADA809149
:10254000E8008B778093E80051CF805DE7CF292F9B
:1025500033272330310509F44EC078F52130310599
:1025600009F488C08BE590E0E8E7F2E0223031051D
:1025700009F03CCF2091E800277F2093E8002091CC
:102580001C0230911D028217930708F49C0140E061
:102590002115310509F073C0411171C08091E80027
:1025A00082FDCDCF8091ED02811549F2853039F25F
:1025B0008091E80083FFF2CFC2CF80911A02909100
:1025C0001B022132310509F446C02232310509F0DF
:1025D0000DCF8330910508F009CFFC01EE0FFF1FEE
:1025E000E15DFE4F0190F081E02D845D9E4FDC01A6
:1025F0008C9190E010C09C013327823021F1233070
:10260000310568F4232BB9F4E7E2F3E0E4918E2F6F
:1026100090E0E7E2F3E0009709F4E8CEABCF233097
:10262000310509F0E3CEE5EEF2E0E4918E2F90E083
:10263000E5EEF2E0F0CFE1E1F3E0E4918E2F90E0FF
:10264000E1E1F3E0E8CFE3E0F3E0E4918E2F90E006
:10265000E3E0F3E0E0CF8330910508F0C7CEFC0162
:10266000EE0FFF1FEB5CFE4F0190F081E02D89E043
:1026700090E080CF82E190E0E3EDF2E07BCF8091CB
:10268000ED02811509F45BCF853009F458CF8091B4
:10269000E80083FD54CF8091E80082FD7FCF8091D8
:1026A000E80080FF75CF9091F3008091F200211532
:1026B000310519F08830910550F041E0089709F094
:1026C00040E08091E8008E778093E80061CF4491EC
:1026D0004093F1003196215031090196E8CF8038BE
:1026E00009F084CE8091E800877F8093E800809194
:1026F00014028093F10070CE811178CE10911802EF
:10270000123008F073CE8091E800877F8093E80054
:1027100010931402D7D91115D9F084E08093ED02FB
:1027200042E061EC81E04BDA42E261EC84E047DABE
:1027300042E261EC82E043DA42E260EC83E03FDABD
:102740008091ED02843051F482E0809320014ECEDE
:102750008091E30087FDE1CF81E0E0CF81E0F5CF1C
:10276000CF93DF93EC014A855B856E857F850E9460
:102770009E0A9B8190958091BA0489238093BA0424
:102780008C810E94A105B3DB86E0FE0111928A953F
:10279000E9F7DF91CF910895CF93DF93EC018D811D
:1027A00081FD16C082608D838091BA049B81892B44
:1027B0008093BA048091B8049C81892B8093B804DB
:1027C00096DB488559856E857F85CE010E949E0ADD
:1027D0001092A8041092A7048D8180FD02C0CE0142
:1027E000BFDFDF91CF9108951F93CF93DF93182F11
:1027F000A0911D04B0911E04109709F448C01092D6
:10280000200410921F041092A3031092A2031696A4
:10281000CD91DC911797CE019A9581159F4108F4CF
:10282000D07ED1E0C11101C0D0E01996ED91FC91AC
:102830001A97309731F01B966D917C9180E0099545
:10284000D823D11539F08CEF8C0F813A20F58C2FDD
:102850000E94360B1115A1F0E0911D04F0911E04A9
:10286000808584FD0DC080911C04811549F0808114
:1028700091819C01215031092F333E4708F488D8BB
:1028800036DB10921E0410921D0410921C04DF917E
:10289000CF911F9108952BDB8C2F0DDCDBCF0F9395
:1028A0001F93CF93DF93843030F5653020F54F30A0
:1028B00010F5C42FD0E0CC0FDD1F2EE1629FC00DBC
:1028C000D11D112436E9839FC00DD11D1124CE01E5
:1028D00089960E949534082F10E0102F0027CE0112
:1028E0008A960E9495349801282BC901DF91CF91D7
:1028F0001F910F91089580E090E0F8CF462F672F49
:102900002091F0023091F102232B81F4703F39F4D1
:10291000403F61F48091EE029091EF02089575308E
:1029200028F44F3018F4843008F4B9CF80E090E0F8
:102930000895A0E0B0E0EFE9F4E10C94A4337C0149
:102940000091700580916F05082BC3E0D0E010E086
:10295000C8010C2E02C0959587950A94E2F780FD78
:1029600009C02197A8F7D12C8D2DCDB7DEB7E7E0B0
:102970000C94C033DC2EB7018C2FC0DF0E94A70659
:10298000019779F3F1CF0F931F93CF93FC018781C8
:102990009085009789F4858100811181811581F0EE
:1029A000611571F0C801C5DFC82F682FC8010E94EA
:1029B000F304B8018C2FA2DFCF911F910F910895DE
:1029C000C8010E942905C82FF4CFCF93DF93D82FD9
:1029D000C92FAFDF6D2F7C2F91DF0E94A706DF91FB
:1029E000CF910895FC0184818115B1F08781908594
:1029F0000097A1F00E94A706282F92959F7096300D
:102A0000B9F080F4925F9F70923030F4203FD1F0A3
:102A100058F481E0283E58F080E00895808191814B
:102A2000D4DFEACF9A5FEFCF81E0243FA9F7089582
:102A300091E0813F09F090E081E0283E08F080E0DD
:102A4000892B089581E00895382F292FCB01A32FDA
:102A5000B22F8F389105A105B10520F48F589C4FF6
:102A60000C94953480E0089585E290E00E949534BE
:102A7000833789F486E290E00E9495348E3B59F4C6
:102A800087E290E00E94953491E08C3F09F090E05D
:102A9000892F8170089580E0FCCFA0E0B0E0E3E5ED
:102AA000F5E10C94A233EC018881811509F18130A4
:102AB00009F045C08981813051F48A81239660E50F
:102AC00070E0893311F060E070E020DBEDCF823000
:102AD00021F48A81239671DAE7CF833021F48A8149
:102AE0002396E9DAE1CF843041F022968111DCCFE0
:102AF000CDB7DEB7E9E00C94BE338A81239620E09F
:102B000030E09AE0682F6053770BAB016A307105B3
:102B100060F02115310551F3EFE9FFE03197F1F74E
:102B200000C0000021503109F4CF929FB001939F63
:102B3000700D11249A01260F371F8991E3CFE82FDA
:102B4000F0E0E850FE4FB490282F26952695269564
:102B500030E0F901E851FE4FE4908770F12C082E27
:102B600002C0F594E7940A94E2F7E0FAEE24FF2419
:102B7000E0F8F901E852FE4FC490D12C082E02C0B3
:102B8000D594C7940A94E2F7C0FACC24DD24C0F8A7
:102B9000F901E853FE4F049110E002C01595079526
:102BA0008A95E2F701701127E114F10411F081EE2A
:102BB00004DAC114D10411F086EEFFD960E070E0B0
:102BC0008B2DA4DAC114D10411F086EE74DAE1146D
:102BD000F10411F081EE6FDA0115110521F060E0CA
:102BE00070E08CE293DA21965FCFAAE0B0E0EBEFE1
:102BF000F5E10C949E33C090EB02D090EC0281E0A2
:102C000090E09093EC028093EB02812C912C10E0E9
:102C1000540100E019C021E030E0133021F0F70149
:102C2000859195919C01472D602F812F39D97394FF
:102C300022E0E20EF11C3FE07312EDCF0F5F8FE058
:102C4000A80EB11C053049F0C501880F991FFC0181
:102C5000E55DFC4F7F01712CDECF1F5FFBE48F0E23
:102C6000911C1430A9F61A8219821C821B821E82C2
:102C70001D8218861F8288EC90E09A87898701E878
:102C800012E09E012F5F3F4F79014AE050E0B8010A
:102C9000C7010E94D434065F1F4F013D32E0130785
:102CA000A1F78AE0F70111928A95E9F74AE050E02E
:102CB000B801C7010E94D434065F1F4F0132F3E010
:102CC0001F07A1F789E0F70111928A95E9F78FEFC5
:102CD0009FEF9E838D8387E08A874AE050E0B801AA
:102CE000C7010E94D434065F1F4F0137F3E01F076E
:102CF000A1F7D092EC02C092EB022A96EDE00C9480
:102D0000BA33AAE0B0E0E7E8F6E10C94A333EFE3CE
:102D1000F2E080E5DF011D928A95E9F7E0ECF4E04E
:102D200088E3DF011D928A95E9F78FE3C82E82E0E0
:102D3000D82E7F0101ED12E0F701D182C0824AE076
:102D400050E0B801CE0101960E94853488E0FE0172
:102D50003196D60101900D928A95E1F789859A8581
:102D6000D70113969C938E931297BAE0CB0ED11C89
:102D7000E7E0EE0EF11C065F1F4F0132F3E01F0784
:102D8000D9F62A96E8E00C94BF33AAE0B0E0EBEC69
:102D9000F6E10C94A13304EA13E081E2E82E83E02B
:102DA000F82E97E0B92E2EE3C22E22E0D22EAA24CE
:102DB000A3944AE050E0B701CE0101960E94853409
:102DC000F8013896DF018B2D1D928A95E9F78981EC
:102DD0009A81D80111969C938E938F8112968C9331
:102DE00012978D8113968C931397888514968C93E4
:102DF0001497898515968C9315978B819C811796CE
:102E00009C938E9316978A8587FD04C01E96DC924C
:102E1000CE921D9780FF02C0F801A08681FF07C0F7
:102E2000D80118969C911897926018969C9382FFEF
:102E300004C0F80190859460908783FF07C0D80193
:102E400018969C911897986018969C9384FF04C0DC
:102E5000F80190859061908785FF07C0D80118968A
:102E60008C911897806218968C93BAE0EB0EF11C47
:102E7000015F1F4FE1E7EE16E3E0FE0609F099CF90
:102E80002A96EAE00C94BD33282FCB01283070F449
:102E90004AE0249F90011124B9016F577D4F4AE009
:102EA00050E00E94853480E090E008958FEF9FEF1E
:102EB0000895AAE0B0E0EFE5F7E10C94A9339C0196
:102EC00097558115914068F4BE016F5F7F4F822F47
:102ED000DBDF892B31F489859A852A96E2E00C9410
:102EE000C53388EC90E0F9CFA0E0B0E0EAE7F7E185
:102EF0000C94A433162FD72FC42FD22E8115A1F0F6
:102F00004093AB040E94650B9093120280931102D0
:102F1000C77081E001C0880FCA95EAF73CD8CDB7E9
:102F2000DEB7E7E00C94C0339091AB04491335C091
:102F3000E0901102F09012020E94650B9C012E1984
:102F40003F097901812F9D2FB4DFE816F90628F596
:102F5000D0E2DD0DCD1591F0C77011E0812F01C0D9
:102F6000880FCA95EAF7E8D8D83040F48D2D8770DD
:102F700001C0110F8A95EAF7812F0DD860E070E04B
:102F8000802FC4D8D83058F62D2D277081E001C08D
:102F9000880F2A95EAF7D0D8C2CFC77081E001C068
:102FA000880FCA95EAF7F7CFA0E0B0E0EAEDF7E1C5
:102FB0000C949D33FC018280648081E08483EDEE7B
:102FC000F4E09490ECE6F5E0E4910091B20406950B
:102FD000015810E0000F111F012F1127C7E9D2E09F
:102FE000C12CD12CAA24AA94B12C77247A94E91963
:102FF000EE2EF12C83E0881630F48091B0048883A3
:103000008091B1048983611017C01B821A829601D6
:103010004A81698188810E9446088FEFC81AD80AC0
:10302000259685E0C816D10429F70E946208CDB71D
:10303000DEB7EEE00C94B9338B818115E9F0815055
:103040008B83789EC00111246C8170E00E946533EF
:10305000FB01FF27E351FB4F8491E82FE9197E9E86
:10306000C0011124B7010E9465338091B204689FAA
:10307000B00111247A83CBCF0E944D34B5010E9458
:103080007933801791071CF683E0881688F00E9438
:103090004D34B5010E94793388830E944D342091CC
:1030A000B1042695622F70E00E947933280F29839E
:1030B0001A828091B204893C20F088EC8C838B8347
:1030C000A6CF8431D8F784E1F9CF0F93CF93DF9364
:1030D000CFEAD4E0488159816A817B8188E090E021
:1030E0000E94C834288139814A815B816C817D814D
:1030F0008E819F8100E20E94EB33622F83E290E099
:103100000E94B634DF91CF910F910895EFEAF4E079
:1031100085E0808311828FEF828383831482CF01C5
:10312000D4CF8091B304833018F48F5F8093B304BD
:103130008FEA94E0CACF8091B304811519F08150D1
:103140008093B3048FEA94E0C0CFA0E0B0E0EBEA54
:10315000F8E10C949E33182FF62E042F722E9091C6
:10316000AF0490FF23C0292F26952695E22FF0E08B
:10317000E55CFE4F80818093AD049C7F9430D9F450
:10318000612F7F2D842F0E94BF07962F672F482F16
:10319000892F0E9477081093B004F092B104009335
:1031A000B204711419F08FEA94E08FDFCDB7DEB767
:1031B000EDE00C94BA33823019F40091B204EBCFF5
:1031C000863019F41091B004E6CF8930D9F38831F4
:1031D00011F7E8EEE20F2170E22EE695F0E0E35100
:1031E000FA4FE491CE2FD0E0A12CB12CC12CD12CE0
:1031F00085E0882E912CC501B4010E946533812F92
:10320000E11012C0860F9601402F6F2D0E944608D4
:103210008FEFC81AD80AAC0EBD1E85E0C816D104BF
:1032200051F70E946208B7CF861BEDCFEFEAF4E0BA
:10323000818121E043816281885F87CFEFEAF4E0FA
:10324000818121E04381628188507FCFEFEAF4E001
:10325000628121E1620F08F46FEF21E043818181F7
:1032600074CFEFEAF4E0628121E1621B08F460E0D0
:1032700021E04381818169CFEFEAF4E0438121E1DC
:10328000420F08F44FEF21E0628181815ECFEFEAC7
:10329000F4E0438121E1421B08F440E021E0628137
:1032A000818153CF9091AF0490FF2CC0811559F1CB
:1032B000893258F58F73880F880F9091AF049370FF
:1032C000892B8093AF04611519F08FEA94E0FDDE3D
:1032D0006091AF046695669570E04BE050E086E043
:1032E00091E00E946434892B91F01092AE0481E049
:1032F0008093D50220E04091B2046091B1048091A6
:10330000B00423CF089581E0D6CF88E2D4CF81E006
:103310008093AE040E94650B9093D3028093D202F7
:10332000E6CF8091AF04869586958F5F893208F04D
:1033300081E061E0B7CF8091AF04869586958A954C
:1033400009F488E261E0AECFACE0B0E0EAEAF9E18E
:103350000C949A337C01DC0114968C91811509F44C
:1033600085C161E0C7010FDB8C01F7018581811503
:1033700021F18091A7049091A8040097F1F008171B
:103380001907D9F0FC01FF27887F9927892B09F0BD
:1033900072C074E0EE0FFF1F7A95E1F7E95DFB4F15
:1033A00085818460858311830083CF01F5D91092D4
:1033B000BA0461E0C701E7DA8C01D70115968C9158
:1033C000811509F4E1C0C80197578038910508F0CC
:1033D0000CC1003108F039C16EE870E080E090E087
:1033E00033DB811132C1812C912C5401011146C073
:1033F00004E09E012F5F3F4F6901D601E02F1D922F
:10340000EA95E9F724013501FFEF4F1A5F0A6F0AC9
:103410007F0AC501B40118DB8983811509F415C140
:10342000813009F0AEC0A50194012E5F3F4F4F4F90
:103430005F4F2D833E834F835887C301B20104DB66
:10344000182F8A83811509F400C18FEF810F833013
:1034500068F56D817E818F819885F6DA8B83811581
:1034600011F0C6011ADB2401350133E0430E511C73
:10347000611C711C49C0E0E0F0E092CFBFE88B1600
:103480009104A104B10409F4E0C0C501B401DCDA7F
:10349000EFEF8E1A9E0AAE0ABE0A8111EFCF0150DD
:1034A000A5CF4D805E806F8078842EC08BEF810F1A
:1034B000833098F52401350143E0440E511C611C12
:1034C000711C6D817E818F819885BEDA8B83811519
:1034D000D9F0C301B201B8DA8C83811571F08B8108
:1034E0009C8181305FEF950710F0982F8827163068
:1034F00071F0173079F00E948C272401350134E0F7
:10350000430E511C611C711C5301420176CF0E9475
:103510003927F3CF0E945A27F0CF143009F0C1CFDA
:103520006D817E818F8198858FDA182F2401350176
:1035300084E0480E511C611C711CC501B4016D5F13
:103540007F4F8F4F9F4F80DA111509F47EC0811590
:1035500009F47BC08150990B4FEF489F9001499F20
:10356000300D1124A12FA150BB0B2A0F3B1F21505E
:10357000310950F2EFE9FFE03197F1F700C00000A8
:10358000F6CFC6018ADAC0CF680127E5D21AC11486
:1035900031E0D30650F568E973E08C2D75DC892B9A
:1035A00021F5C60154E0880F991F5A95E1F7FC01F7
:1035B000E95DFB4F2281213099F5209198033091EC
:1035C0009903232B91F020919A0330919B03232B95
:1035D00061F020919C0330919D0340919E03509196
:1035E0009F03242B352B232B19F1D70115963C90E3
:1035F000311409F43FC00E35BCE71B0719F10F3534
:10360000ECE71E0741F00D35FCE71F0799F58091A7
:1036100021018115B9F01092210180E0E5D815C093
:10362000223019F720919C0330919D03232BE9F25E
:10363000FC01E45DFB4F20812E7F2083895D9B4F41
:10364000ABD8D3CF81E0809321018091BB048770F8
:10365000811561F0D70115968C91811539F0809113
:10366000720582FF03C082E00E9486052C96E1E18C
:103670000C94B63380912101811168C0C80197551F
:103680008115914008F0FEC05801F8EFAF22BB242D
:10369000A114B104D1F6F801FF2734E0EE0FFF1FAB
:1036A0003A95E1F79F01295D3B4F6901D7011596D6
:1036B0008C91E45DFB4F908180FB90F990838115A4
:1036C00009F4D9C10E94650B9093AA048093A904C0
:1036D000F60182818F5F82838091BA049091B80451
:1036E000892B83838091B7048483468157816685C3
:1036F0007785C6010E949E0AD60115968C9181FF9E
:103700005801B092A804A092A704D70115969C91E5
:10371000911509F4E2C51092AB0498013057233299
:10372000310508F0E8C584E090E00E94A23490934F
:10373000720580937105F801E150F047E232F1051E
:1037400008F0E1C1E959FA4C0C948C33380130EEA1
:10375000631A71085090B9048091B804582A809176
:10376000B704582A48E06416710408F05EC0980156
:103770002770332781E090E001C0880F2A95EAF78F
:10378000311409F44FC0582AD7018D919C910E94A1
:10379000290521E030E0F90102C0EE0FFF1F8A95F4
:1037A000E2F7FE83ED8320911D0430911E043A87D9
:1037B000298740912504509126045C874B8744EA71
:1037C000C42E43E0D42EA12CB12C511005C0D6013B
:1037D00012968C9181111BC0F601838190E02D819E
:1037E0003E8182239323892B91F08085982F9770B7
:1037F000911101C087E038E06316710408F066C0DB
:10380000311409F45FC086958170811164C09FEF07
:10381000A91AB90AAFE0CA0ED11CB8E0AB16B104C0
:10382000A1F61CC080955822AFCF311038C08091CE
:103830002504909126040817190781F41092260494
:103840001092250410922104109222041092230455
:10385000109224041092200410921F0480911D04E1
:1038600090911E04009709F409CFE8E06E167104E8
:1038700008F0EBC0652D0E942A0A811103C081E087
:103880000E94F413F7018581F801E851FC47E73005
:10389000F10508F03ACFE757FA4C0C948C331093AB
:1038A0002604009325040E94BC0C609321047093AD
:1038B00022048093230490932404109220041092F5
:1038C0001F0462CF82FB882780F99FCF311409F44F
:1038D0009ECF80FF9CCFD6018D909C900815190536
:1038E00019F4311409F493CFE985FA85EC15FD0537
:1038F00009F48DCFD6011D96ED91FC91309721F002
:103900008081811509F483CF652DC6010E942A0AA2
:10391000811509F47CCF81E00815190509F080E0D4
:10392000482E43208114910441F0411006C0EB85DC
:10393000FC858E169F0609F06ACF80E00E94F41382
:10394000D0921E04C0921D0481E080931C048FE07D
:103950008A9DF0018B9DF00D1124EC55FC4F858163
:103960008093A30341100EC08114910459F080810B
:1039700091819C0124503109213A310508F049C058
:103980000E94360B8FE08A9DF0018B9DF00D112473
:10399000EC55FC4FC680D780C6019A9581159F4192
:1039A00010F420EED22299249394C60101978F330C
:1039B0009E4708F0912C8FE08A9DD0018B9DB00D21
:1039C0001124AC55BC4F1996ED91FC911A97309784
:1039D00031F01B966D917C9181E0099598229114AC
:1039E000A9F08FE08A9DF0018B9DF00D1124EC551C
:1039F000FC4F868197810E94A2048093A203C60196
:103A000048E06416710440F40E94C80C0E94770FCD
:103A10000AC00E945B10B6CF0497813A910548F422
:103A20008C2D0E94020B411409F428CE0E94770FBE
:103A30000CCE0E94770F8FE39CE90197F1F700C04D
:103A400000008C2D0E94DD0FEECFDC012D913C910A
:103A50000217130741F4311009C010921C0480E0D2
:103A60000E94F4130BCE311409F408CEFC018085BA
:103A700085FD04CEF4CFF9014485558566857785AB
:103A8000C9010E949E0AD60115968C9181FF3DCEF8
:103A9000C6010E94B0138091A7049091A804081752
:103AA000190709F032CE1092A8041092A7042DCE67
:103AB00006E221EE41EE6AE17CE716DAC6CD07E2C6
:103AC00025EE45EE6BE17CE7F8CF06E221EE40EE15
:103AD00068E17CE7F2CF07E225EE44EE69E17CE79E
:103AE000ECCF06E221EE42EE6CE17CE7E6CF07E2A6
:103AF00025EE46EE6DE17CE7E0CF08E221E045EE01
:103B00006EE17CE7DACF8091710581608093710569
:103B1000609171057091720584E090E00E94D0344C
:103B20000E94AC1092CD80917205886080937205DE
:103B3000EFCF809171058260E9CF8091710584603B
:103B4000E5CF809171058860E1CF80917205816039
:103B5000EDCF809172058260E9CF8091710580611F
:103B6000D5CF809171058062D1CF8091710580643D
:103B7000CDCF0E94AC10809171058068C7CF809135
:103B800071058C60C3CF809172058360CFCF809127
:103B900071058E7FBBCF80917205877FC7CF8091E3
:103BA00071058D7FB3CF809171058B7FAFCF8091F1
:103BB0007105877FABCF809172058E7FB7CF8091E3
:103BC00072058D7FB3CF809171058F7E9FCF8091DD
:103BD00071058F7D9BCF809171058F7B97CF0E9460
:103BE000AC10809171058F7791CF80917105837FA3
:103BF0008DCF809172058C7F99CF80917105992727
:103C000082FF939590FB82F990FB83F97FCF80919F
:103C10007205982F909590FB80F990FB81F986CFE3
:103C200090917105892F8F7B96FF80646FCF0E94E2
:103C3000AC1090917105892F97FB87F9805866CF5A
:103C400061E08EE090E00E94B63462CF60E0F9CF90
:103C500090917105892F8F7E94FF806157CF90914D
:103C60007105892F8E7F90FF816050CF90917205F2
:103C7000892F877F93FF886059CF89E24EC389E2FD
:103C800037C30737BCE71B0709F053C081E00E9428
:103C9000E50471C08272F801E052F847EB30F1059B
:103CA00008F043C0E057FA4C0C948C338091AF0479
:103CB00080FF0BC08E7F8093AF048FEA94E005DA1B
:103CC0001092AE040E946208C0CC81608093AF0461
:103CD00061E086958695E6DAB8CC811521F02BDB7C
:103CE000B4CC8115E1F31DDBB0CC811521F0A6DA4F
:103CF000ACCC8115E1F39ADAA8CC811521F0B1DAC8
:103D0000A4CC8115E1F3A2DAA0CC811521F0BFDAB1
:103D10009CCC8115E1F3B0DA98CC811521F00BDA57
:103D200094CC8115E1F3FDD990CC0737ECE71E0761
:103D3000F9F00837FCE71F0721F19801205E3245B2
:103D40002032310518F5911138C00F7181E090E0F3
:103D50009C0102C0220F331F0A95E2F78901622FEE
:103D600083E090E00E94B634802F0E94D5046DCC91
:103D700081E00E94DB0443E062E081E00E945D0597
:103D800064CC82E0911509F482CFF3CF9115A9F0AC
:103D90000A353CE7130709F476C008F04EC001303D
:103DA0005CE7150709F46DC003308CE7180709F4C8
:103DB00062C001151C4709F451C0F7018781908545
:103DC000009709F464C00E94A7068C01F701B58032
:103DD000A680A2942FE0A2228091BB048770811557
:103DE00001F1CB2CB114F1F0812F807F803461F090
:103DF00080E2800F8830A8F0812F807E803221F40D
:103E0000023078F0A11469F08091720582FF09C038
:103E100082E00E9486058091BB048770CC24C39405
:103E20008111C12CE12FE295EF70103C08F0A5C084
:103E3000F0E0E556FA4C0C948C330B35ACE71A07DE
:103E400021F180917205002482FF0394802D0C35AE
:103E50001C4709F0B2CF0E94390FAFCF0E94AC10BF
:103E6000EFEFF4E32CE0E150F0402040E1F700C038
:103E700000000E94AE0E6FEF7FEF80E090E00E94A6
:103E8000D0340E94D81081E0E6CF80E0E4CF858175
:103E9000C080D180811569F0C6010E949914182F45
:103EA000682FC6010E94F304B601812F0E947E1480
:103EB0008ACFC6010E942905182FF6CFF12FFF7077
:103EC000DF2E103118F0D29490EFD922B114B9F04E
:103ED000D11469F080E2800F883010F0011109C020
:103EE0008091B8048D298093B8040E94770F802FA9
:103EF00042C08091BA048D298093BA04F6CF802FF6
:103F00000E945B10D114C9F180E2800F883010F05C
:103F1000011104C08D2D0E94A10506C0D09480918E
:103F2000BA048D218093BA040E94770F26C0212FF6
:103F30002F70D22E107F103219F0D29480EFD82239
:103F4000011549F0013009F484C0B11409F490C09E
:103F5000A114B1F1CCCF8091720582FD2DC0B114B6
:103F600029F1D11439F08091B8048D298093B804D7
:103F70000E94770F80E00E94DD0FC11409F4D8C0C1
:103F80008091BB0480FDD4C0D70115961C92869504
:103F9000869586950E94DB04C701D6D98091BB0423
:103FA0008695869586950E94E504C2C080E00E94B1
:103FB0005B10D11411F3AECFB11469F1A11004C09C
:103FC0008D2D0E94CB0FD9CF31E0A31210C01091DC
:103FD000B7048D2D8123D81681F20E94650B909332
:103FE000BF048093BE041D291093B704C6CF45E0DB
:103FF000A412C3CF8D2D0E94CB0F8D2D0E94C30B19
:104000008091B9049D2D9823D91609F4B6CF8D2936
:104010008093B904B2CFA11012C08D2D0E949C10C4
:104020008D2D0E94C30B8091B9049D2D982391156D
:1040300009F4A3CFD094D822D092B9049ECF51E0F6
:10404000A5129BCF8091B8048D21811509F495CFDD
:10405000E4CFB11429F086E0A81608F08ECFB0CFD7
:1040600095E0A91608F089CF8D2D0E949C1085CF70
:10407000A114D1F3093349F4AFEFB7EEE3E0A15057
:10408000B040E040E1F700C00000802F0E945B10CC
:1040900074CF812F869586958370811561F081306C
:1040A00009F06BCFC8019370B11002C080E090E0BE
:1040B0000E94DA0A62CFC8019370B11002C080E09A
:1040C00090E00E94B20A59CF6B2D802F0E94010C04
:1040D00054CF812F8370811138C0B11027C0402F79
:1040E000429546954770440F440F802F8F70042EE1
:1040F00001C0880F0A94EAF7202F207104FF07C03F
:104100002FE030E001C0220F4A95EAF7209516957E
:10411000169513701230A1F0133081F030916F05B5
:10412000113059F0822B83230E94D5040E94A30AE8
:1041300060E0C7010E94C31499CA832B822BF4CF7D
:10414000822B90916F058927EFCFB11451F110FFA9
:10415000EDCF402F429546954770440F440F802F76
:104160008F70042E01C0880F0A94EAF7202F207167
:1041700004FF07C02FE030E001C0220F4A95EAF7A4
:104180002095169516951370123089F0133069F04A
:1041900030917005113041F0822B83230E94D804A6
:1041A000C5CF8230B0F6C2CF832B822BF7CF822BC4
:1041B000909170058927F2CF1F70B11439F0812FCB
:1041C0000E94DB04802F0E94CB0FB0CF802F0E9473
:1041D0009C10812F0E94E504A9CF023F71F170F479
:1041E000003FC9F0013F91F0B11409F465C0A1147A
:1041F00009F45FC0802F0E94DD0F98CF033F21F1AB
:10420000043F91F78091720582FD2AC0812F8F7142
:10421000B11401F316C0B11469F0F5E0AF1608F05F
:1042200085CF1F7181E090E0012E01C0880F0A94B4
:10423000EAF7BECF26E0A216F2CF812F8F71B11020
:10424000C9CF0E94DB0472CF80E0B11409F4A6CF7D
:104250001F7181E0012E01C0880F0A94EAF79ECFFA
:10426000B114C1F08091BB048770843049F410927E
:10427000BB041092BD041092BC04812F8F71AACF91
:1042800035E063E0A31608F051CF812F8F710E94B3
:10429000AF0B4CCF45E0A41640F01092BB04109237
:1042A000BD041092BC0464E0F0CF81E00E9486055A
:1042B0003DCF812F8F71C5CFA114F9F2093349F495
:1042C0005FEF87EE93E0515080409040E1F700C0EF
:1042D0000000802F0E945B1029CF0631BCE71B072E
:1042E00009F0CFCC8091AC04811509F4C8CC85E3EA
:1042F0000E94360B9BCB8091B8040631ECE71E0779
:1043000009F0C8CC8A7A91E0811101C090E09093C5
:10431000AC04811509F4B1CC85E30E94020B86CB75
:10432000A0E0B0E0E6E9F1E20C94A43380916E03E2
:10433000803108F049C080916D03811509F444C0B3
:10434000C0911F0389E0D82E80911E038C17E1F1E4
:10435000EC2EF12CDC9EE0011124FE01E05EFC4F0E
:1043600084818115B1F1918180916903981331C0E5
:1043700090818091680398132CC08581811129C098
:104380000281138180916A0390916B03081B190BC2
:1043900060E088E693E00E94C3140E945917081752
:1043A0001907B8F480916E038F70806180936E035B
:1043B000CA5DDC4F88818F708061888388E693E0D6
:1043C0000E94A4190E947C05CDB7DEB7E7E00C94EB
:1043D000C033E7012196C770B7CFAFE0B0E0E3EF9D
:1043E000F1E20C949C338C0186E0F801DE011A9610
:1043F00001900D928A95E1F7F801F580E48088E656
:10440000882E83E0982E80916C03811117C0E114EF
:1044100091F0F11409F480C1C8010E94F2148115D1
:1044200009F47AC189E0F801A8E6B3E001900D92A1
:104430008A95E1F775DFFF24F3946AC0A280B38008
:10444000D0906D0380916A0390916B033501681AD7
:10445000790AD11409F411C1C080518060E088E666
:1044600093E00E94C3140E9459176816790608F059
:10447000B6C0E11401F380916903F8019181E090E5
:104480006E03F0E1EF1608F064C0981320C090911D
:104490006803F801808198131AC020916F0330914E
:1044A0007003878190852817390789F4F1104BC074
:1044B0008E2D8F70806180936E0388E693E00E945A
:1044C000A41980916E03F8018683F12C21C0F110AC
:1044D0003AC040E0652D8C2D0E94690E40E0652DAC
:1044E0008C2D0E94690EF82E8111EFCF8A859B8555
:1044F0000E94E514292F22952F70903470F49F703C
:104500002230A0F09115B1F0F8019681903190F42D
:104510008F2D2F96EFE00C94B8332A5F2F70223046
:1045200068F0C8010E94A419FD2CF2CF911511F07A
:10453000811571F3805E883058F3F3CF803F40F3EC
:10454000815F8330F9CF80916E03816080936E0329
:10455000BCCF98131EC090916803F8018081981316
:1045600018C020916F0330917003878190852817C0
:10457000390779F4F1100DC0E682C8010E94A41930
:1045800089E0F801A8E6B3E001900D928A95E1F781
:1045900052CFC8010E94F214811509F4BDC0F11474
:1045A00009F4BAC080916E03803208F43BCF809149
:1045B0006803909169039A838983BC82AB8280915E
:1045C0006C038D831E82EF8280916F039091700344
:1045D00099878887CE0101960E94A41923CFD09095
:1045E0006E03F0E1DF1650F488E693E00E94A41910
:1045F00089E0F40111928A95E9F767CFE11409F493
:104600001ACF90916903F801818198131AC0909193
:1046100068038081981315C020916F033091700357
:10462000878190852817390761F4F1100AC0D68276
:10463000C8010E94A41989E0F40111928A95E9F752
:10464000FACEC8010E94F214811509F465C0F11474
:1046500009F462C080916E03803208F4E3CE809149
:104660006803909169039A838983BC82AB828091AD
:104670006C038D831E82DF82A7CF60E088E693E023
:104680000E94C3140E9459176816790608F0B0CF2B
:10469000E11409F4D0CEF11409F43EC090916903FD
:1046A000F801818198132EC090916803808198133E
:1046B00029C020916F03309170038781908528175E
:1046C000390701F580916A0390916B03A81AB90A22
:1046D000F8ECAF16B10408F053CF80916E0380FD63
:1046E0004FCF803108F44CCFF8018683982F907F0C
:1046F000903F09F442CF982F907F905F8F70892B65
:1047000086833BCFC8010E94F21481118BCE809129
:104710006E03816080936E03C8010E94A4198BCE42
:10472000A2E1B0E0E6E9F3E20C94A7330A871B8725
:104730002C873D874E875F87688B798B8A8BCE016C
:104740000A964BDE811128C020911E0330911F0371
:1047500089E0FE013A96DE01119601900D928A954C
:10476000E1F78E858115C1F0822F90E00196877068
:10477000992738171906D9F099E0929FD001112492
:10478000A05EBC4FFE01319601900D929A95E1F723
:1047900080931E030E947C0519E080911F03909175
:1047A0001E03891312C06296E4E00C94C3330E9486
:1047B000AC1010921E0310921F0389E0E8E6F3E0AC
:1047C000DF011D928A95E9F7E7CF189FC0011124F8
:1047D000805E9C4F02DE811531F380911F0390E0D3
:1047E00001968770992780931F03D7CFEF92FF928E
:1047F0000F931F93CF93DF9380916C05E0912E026E
:10480000CDE0811130C0CDB7DEB7E6E00C94C13306
:10481000D1E0DE0FD0932E02EE2EF12CCE9FF001D0
:104820001124EC5FFA4F84818115E1F08781908536
:10483000892B21F481859285019651F400811181A3
:10484000228133814481558166817781808568DF4B
:10485000CE9DF001CF9DF00D1124EC5FFA4F148234
:104860001092BA04ED2F80916C05E81788F210922F
:104870006C0510922E02C7CFA4E0B0E0E2E4F4E2AF
:104880000C949A3320910305298397E0992E01E037
:1048900010E02DE0322E34E0532E88248394809152
:1048A00002059981891307C0A1DF0E94ED092496B2
:1048B000E1E10C94B6339981892F90E09C838B833E
:1048C000FC01EE0FFF1FE850FB4F80819181989E05
:1048D000D001999EB00D1124FD01E054FB4FFA83E5
:1048E000E983248121115BC060906C05E4E0F5E070
:1048F00060E070E0712C661508F04FC0A384B484AA
:10490000A981BA81CD90DC902FEF3FEF412C442D4F
:1049100050E07601E40CF11CE40CF11CD701ED90A1
:10492000FC90E114F10439F0AE14BF0409F0A901C0
:1049300043949A01ECCF2F3F3207D1F1D80102C046
:10494000AA0FBB1F2A95E2F77A2A9801042C02C00D
:10495000220F331F0A94E2F7A9014150510974163E
:10496000150629F5369EF001379EF00D1124EC5FF7
:10497000FA4F989ED001999EB00D1124A054BB4FC0
:1049800012962D913C911397308727835482108281
:1049900011829287818715968C920E94FE098B81E5
:1049A0009C8101969A8389838370898378CF14824E
:1049B0006F5F7F4F3D969FCF10926E0510926D05F1
:1049C0001092220180910205809303050E94ED0957
:1049D0000DCFACE1B0E0EFEEF4E20C9499334B8BE9
:1049E0005C8B6D8B7E8B8F8BB92E988FA92E91113E
:1049F0001092BA04188A198A1A8A86E0FE01739600
:104A0000DE011A9601900D928A95E1F75F888091F8
:104A1000720582FF1FC00E94650B2091BC0430917B
:104A2000BD04821B930B8838934138F08091BB04FE
:104A300082FD03C082E00E9486050E94650B2091E2
:104A4000BE043091BF04821B930B8838934110F051
:104A50000E94A9055114D9F05E86BF8661E0CE019F
:104A60000A960E94C31461E0CE010A960E94C31404
:104A700061E0CE010A960E94C3144C0180356CE7B8
:104A8000960791F4A11419F181E0809322015E86CA
:104A9000BF860A851B852C853D85452D5B2D688944
:104AA00079898A893DDECDC081359C4721F4A114E6
:104AB00071F082DFECCF82E588168CE7980639F436
:104AC000A11429F0809122018111F3CFDDCF40ECB8
:104AD000E42E44E0F42E412C612C712CD7016D9111
:104AE0007C91CC24CA94DD24DA9480E0282F30E035
:104AF000FB01E80FF11DE80FF11D408151814115C7
:104B0000510539F08416950609F096018F5F690109
:104B1000EDCF10E0BFEFCB16DB0609F44EC0F70176
:104B2000448110912201411110E0D70115963C906B
:104B3000159716969C911697A11409F405C11115A5
:104B400009F402C1311017C021E030E00C2C01C083
:104B5000220F0A94EAF7922B16969C932091000557
:104B6000309101052233310530F422E330E03093F7
:104B7000010520930005E1E0F0E002C0EE0FFF1F09
:104B80008A95E2F7CF010197D70116962C91281745
:104B9000190699F4C0906D05D0906E05C114D1042A
:104BA00009F453C00E94650B8C199D09C39708F442
:104BB0004CC081E0F701848311E0412ABFEF6B1AFA
:104BC0007B0AE7E0EE0EF11CF8E06F16710409F0C5
:104BD00085CFA11409F417C1411409F414C10E942E
:104BE000650B90936E0580936D0580916C05883000
:104BF00040F591E0980F90936C0599E0FE013A968C
:104C0000DE01119601900D929A95E1F75D82BE82C8
:104C10002DE0829FC00111248C5F9A4F29E0FE0194
:104C20003196DC0101900D922A95E1F72FEF3FEFCD
:104C3000DC011A963C932E9319971C969C928E92A7
:104C40001B976C96E2E10C94B5332091030580919B
:104C50000205922FE0E0F0E001E0281709F448C0D7
:104C6000422F50E0FA01EE0FFF1FE850FB4F20806B
:104C7000318037E0329DF001339DF00D1124E05476
:104C8000FB4F608171817C8F6B8FB0E030E0A0E0E2
:104C9000EB8DFC8DEA0FF11DEA0FF11DC080D18074
:104CA000C114D104E1F0F7010190F081E02DFA8FF9
:104CB000E98F30E007C0E1E0C616D70609F0E0E072
:104CC000BE2B3F5FE98DFA8DE30FF11DE30FF11D60
:104CD000608171816115710571F7AF5FD9CFB11531
:104CE00081F13A17C8F4E1E0D7011496EC93F7018B
:104CF00090930305EE15FF0509F45FCF90E0FC01EA
:104D0000EE0FFF1FE850FB4F7182608201968370A7
:104D100099278093020551CF37E0329DF001339DF2
:104D2000F00D1124E054FB4F0483EE15FF05F9F25A
:104D3000291302C09F5F93709A012F5F3F4F23702A
:104D40008CCFE0E0F0E0F8CF292F30E0311024C024
:104D500061E070E002C0660F771F8A95E2F7CB0131
:104D600001972817390791F010E0E1E0F0E002C068
:104D7000EE0FFF1FCA94E2F76F01C094D701169699
:104D80008C9116978C2116968C9317CF411569F349
:104D9000C3010E94FE09E8CFA9010C2C02C0559561
:104DA00047950A94E2F7C901019782239323892B3F
:104DB00039F540FF25C0D70112968D919C91892B22
:104DC000D1F087E0FE013196DF011D928A95E9F767
:104DD0000E94650B9C018B839C8384E08D83F7018B
:104DE00092818381792F9887898709811A8144E08C
:104DF0005E816F8195DCD70115961C92132DB5CF7E
:104E0000142F1170B2CF909103058091020598176D
:104E100031F032DDB1E04B1609F413CF38CEE6DCC9
:104E200010926E0510926D050E94ED09F3CFA6E079
:104E3000B0E0EDE1F7E20C94A7330E94650B8C0122
:104E40008091F2029091F3028017910771F019821C
:104E50001A820E94650BBC0149815A8180E090E072
:104E6000B8DD1093F3020093F2022696E4E00C946E
:104E7000C333A6E0B0E0EFE3F7E20C94A9339093DC
:104E8000EF028093EE02811520E2920730F40E9437
:104E900046102696E2E00C94C53380EF89838A831E
:104EA0000E94650B8160BC0149815A8181E091E0DB
:104EB00090DDEFCFA6E0B0E0E0E6F7E20C94A73398
:104EC0008C019093EF028093EE02011580E21807A7
:104ED000B0F4802F0E945B10C801805E9109089792
:104EE00028F062EA70E10115110511F46CE970E136
:104EF000C8010E94CC042696E4E00C94C33380EFF2
:104F000089838A830E94650B8160BC0149815A8133
:104F100081E090E05EDDEFCFCF93DF93D82FC92FF4
:104F2000A8DF8D2F9C2FC6DFDF91CF9108950F93BF
:104F30001F93CF93DF938C01862F68E973E00E9463
:104F40004417892B91F4C0919803D091990320972D
:104F500061F0F8018281833039F4CE01DDDFCE01CA
:104F6000DBDFCE01D9DF01C0E0F7DF91CF911F91E8
:104F70000F9108950F931F93CF93DF938C01EB0153
:104F800068E973E08C2F0E944417892B09F057C001
:104F9000FE01FF27D80112968C911297E157FD4F21
:104FA0008130A9F415968C9182FD4EC080FF4CC0D3
:104FB00082E0808380919A0390919B030097B9F4DB
:104FC00080919803909199030097C9F110C08230A5
:104FD000A1F515968C9182FD26C080FD0AC083E064
:104FE000808380919C0390919D030097F1F041DFB5
:104FF00026C084E0808380919E0390919F03009758
:10500000B1F78091980390919903009701F184DFA3
:1050100080919A0390919B03009749F780919803A0
:1050200090919903E4CF85E08083809198039091DB
:105030009903009721F070DFF1CF86E08083DF9144
:10504000CF911F910F91089581E08083B9CF809116
:105050009A0390919B03B8CF0F931F93CF93DF9345
:105060008C01EB0168E973E08C2F0E944417892BB7
:1050700071F4DD27C157DD4F8881F8011282188253
:105080008330E9F048F4813059F0823081F0DF91CB
:10509000CF911F910F9108958430B1F08530B9F709
:1050A0008091980390919903009789F306C08091AD
:1050B0009A0390919B03009799F3FCDEE8CF8091CF
:1050C0009C0390919D03F7CF80919E0390919F0345
:1050D000009799F7209198033091990380919A0352
:1050E00090919B0321153105F9F2009731F7C90121
:1050F000E4CFA0E1B0E0EFE7F8E20C949B33FE01CF
:10510000319680E1DF011D928A95E9F709E010E010
:1051100091E7A92E93E0B92E2FE8422E512C612C55
:10512000712C4F0173016201B1E14B16510461040E
:1051300071041CF080E1C82ED12CA601B501C40178
:105140000E94A734AC0CBD1C0D2C000CEE08FF080F
:105150004C185D086E087F080150104019F76096E2
:10516000E0E10C94B7336FEF85E290E00E94B63433
:105170006FEF86E290E00E94B6346FEF87E290E036
:105180000E94B63460E088E290E00E94B6340E944B
:10519000F515AFDF63E785E290E00E94B6346EEB71
:1051A00086E290E00E94B6346CEF87E290E00C94C7
:1051B000B6348F929F92AF92BF92CF92DF92EF92CE
:1051C000FF920F93CF93DF9388E090E00E949D348D
:1051D0004B015C01CFEAD4E068839982AA82BB824A
:1051E0001C821D821E821F8283E290E00E94953401
:1051F000282F30E040E050E060E070E080E090E098
:1052000000E20E94D033282939294A295B292883C2
:1052100039834A835B836C837D838E839F83DF9195
:10522000CF910F91FF90EF90DF90CF90BF90AF9014
:105230009F908F900895AAE0B0E0E1E2F9E20C942B
:105240009D33FE0131968AE0DF011D928A95E9F7D0
:1052500094E6A92E91E0B92E8F013F01EE24E3944C
:10526000F12C38E7C32E31E0D32EF50181915F0197
:105270008F3F09F444C0F894E82FE295EF70F0E016
:1052800021A18F70A70102C0440F551F8A95E2F734
:10529000CA01922F982B91A392A18095892382A372
:1052A000789400C0E9E6F1E021E030E0812C912C17
:1052B00041914F3F79F0A42FA295AF70A05EB0E06E
:1052C0008C9190E04F7002C0959587954A95E2F7D2
:1052D00080FF3BC080E090E0882A992A220F331F8C
:1052E000CE16DF0629F7F50182918F3F11F00E945B
:1052F000A50750EA5A95F1F7D8018D929C920E5F5E
:105300001F4FB9E6AB16B1E0BB0609F0AECF4AE0DD
:1053100050E0B30182EB92E00E947134892BB9F026
:105320008AE0F301A2EBB2E001900D928A95E1F7D9
:1053300081E0809310020E94650B90930F0280938E
:105340000E022A96EEE00C94B933C901C5CF8091C4
:1053500010028115B1F300910E0210910F020E940C
:10536000650B801B910B059760F34AE050E062EB00
:1053700072E081EE92E00E947134892B49F08AE05C
:10538000E2EBF2E0A1EEB2E001900D928A95E1F736
:1053900010921002D6CFCDB7DEB7AC970FB6F89407
:1053A000DEBF0FBECDBF85B7806885BF85B780687B
:1053B00085BF84B7877F84BF0FB6F894A895809186
:1053C0006000886180936000109260000FBE80E8EA
:1053D00090E00FB6F89480936100909361000FBE47
:1053E00081E08093200183EA97E09093E501809328
:1053F000E4010E94C8090E9481160E94C5160E94FD
:10540000B20D0E940F0E8091E20084608093E20052
:1054100078948091ED02811599F08091E9001091C6
:10542000EC008F70179511271795182B1092E90033
:105430008091E80083FD0E94ED101F701093E90039
:1054400082E084BD93E095BD9AEF97BD80936E0096
:105450000E943415811101C086DE04E611E0D801F6
:105460008D918D018F3F11F00E94A507B1E00936A3
:105470001B07A9F709E611E0F80181918F018F3F21
:1054800011F00E94A507F1E008371F07A9F78AE08D
:10549000E1EEF2E0DF01282F1D922A95E9F7E2EB19
:1054A000F2E0DF011D928A95E9F780E090E00E942A
:1054B000A234833E9E4F21F40E94341581112AC0EC
:1054C00063EE7EEF80E090E00E94D03460E082E006
:1054D00090E00E94B63481E080936F0561E083E044
:1054E00090E00E94B63460E074E184E090E00E94B5
:1054F000D0340E94861837DE40E050E0BA018FE0D9
:1055000090E00E94C83440E050E0BA0183E190E0AE
:105510000E94C83482E090E00E9495348093BF02DC
:1055200084E090E00E94A23490937205809371050C
:1055300082DEEFEFF6E721E0E150F0402040E1F7B6
:1055400000C0000078DE8091E10280FF08C06FEFAC
:105550007FEF80E090E00E94D0340E94AE0E83E0A6
:1055600090E00E9495340E94D5048091BC02811184
:105570001EC08FEA94E01DDE8091AF04843028F4D1
:105580000E9486188FEA94E014DE0E94540810925C
:10559000AE040E94E0098091AF0480FF05C060E086
:1055A000869586950E94521981E08093BC0281E124
:1055B00091E090931503809314038091ED0210E421
:1055C000853009F48AC037DE60ECA62E62E0B62E84
:1055D00001EE12E0D801F501219131918D919D915B
:1055E00042E0EA3CF40709F482C028173907A1F326
:1055F00051EE852E52E0952E512CD401ED90FD9068
:105600004D01F501619071905F016E147F0451F1BD
:105610006E247F24412CCC24C394D12CC3018C2133
:105620009D21892BB1F049825A820E94650B9C838F
:105630008B83F1E0FD8391E097012C213D21232B09
:1056400009F490E09E8349815A816B817C818D8130
:10565000C0D94394CC0CDD1C2FE04212DFCFF50102
:10566000F292E292539435E05312C7CF0E94BC0CE1
:1056700043C08091ED02843019F11092BD0288E19F
:1056800090E00FB6F894A895809360000FBE109339
:10569000600083B7817F846083BF83B7816083BFED
:1056A0007894889583B78E7F83BF0FB6F894A895BA
:1056B00080916000886180936000109260000FBE4E
:1056C000BADDE1EEF2E081919191892B09F049C6B2
:1056D000ABEEB2E0AE17BF07B1F78091ED028530B7
:1056E00009F4C7CF0E94AC100E94A30A6CCF281700
:1056F000390709F07DCF9BDBE0901F04F090200478
:10570000E114F10491F18090CE029090CF02A0902C
:10571000D002B090D1020E94BC0C681979098A09A4
:105720009B098090CA029090CB02A090CC02B090CE
:10573000CD02681579058A059B05B8F0C7010E945E
:1057400046101092200410921F041092CE02109264
:10575000CF021092D0021092D1021092CA0210927F
:10576000CB021092CC021092CD02C090A704D09030
:10577000A804C114D10439F1A090A904B090AA04DE
:105780000E94650B7C01EA18FB08C6010E945917AC
:105790008E159F05C0F42091A7043091A804C9017B
:1057A0009927287F3327232B09F08FC124E0880F06
:1057B000991F2A95E1F7895D9B4FDC0115962C9185
:1057C00022FF0E94CC1380912201811511F1E090FB
:1057D0006D05F0906E05E114F104D9F00E94650B9F
:1057E0008E199F092091000530910105281739076E
:1057F00080F49091030580910205981709F468C11F
:105800003BD8109201051092000510926E0510927F
:105810006D058091AE04811509F444C08091AD04FA
:10582000E091AF04E695E695E81BE093D4028F3053
:1058300009F495C108F055C1863009F479C1893061
:1058400009F481C1823009F468C180EDE82E87E057
:10585000F82E9EEBC92E97E0D92E8091D5028115A6
:1058600061F01092D5020E94650B9093D302809351
:10587000D2021092D7021092D6020E94650B20919C
:10588000D2023091D302821B930B8F3F9F4750F47B
:105890002E0D3F1D3093D3022093D20282ED92E071
:1058A000F601099586E0E2E9F3E0DE011196019048
:1058B0000D928A95E1F790909303B0909403F09045
:1058C0009503A0909603E090970310929403109292
:1058D000950310929603109297038F2D8B298115B3
:1058E00009F441C0C090DA02D090DB020E94650B3F
:1058F0009C012C193D0990919003911509F42CC538
:105900002531310580F19F3F19F09F5F90939003FF
:10591000B11459F00E94590A91E01B140CF09FEF4A
:10592000899F802D112480939403F11459F00E94D3
:10593000590A91E01F140CF09FEF899F802D1124CC
:105940008093950380919403811569F0D09095031D
:10595000D11449F00E944B0A809394038D2D0E942C
:105960004B0A809395038A2D8E29811509F441C035
:10597000C090D802D090D9020E94650B9C012C19CE
:105980003D0990918F03911509F4E1C4213531054A
:1059900080F19F3F19F09F5F90938F03A11459F0FE
:1059A0000E94790A91E01A140CF09FEF899F802DD4
:1059B000112480939603E11459F00E94790A91E032
:1059C0001E140CF09FEF899F802D11248093970364
:1059D00080919603811569F0D0909703D11449F016
:1059E0000E944B0A809396038D2D0E944B0A809350
:1059F000970380919303891119C0809194038115B5
:105A000011F08B1113C020919503211511F02F1166
:105A10000DC090919703911511F09E1107C0309120
:105A20009603311103C0822B892B81110E94D80B60
:105A300086E0FE013196A2E9B3E001900D928A95CD
:105A4000E1F70E94A30A9091DC02891721F080936C
:105A5000DC020E94BC0C8091ED02843009F0ADCDD7
:105A600083E08093E9008091E80082FFA6CD8091D9
:105A7000E80090E085FF06C00E94810D811509F4C1
:105A800089C091E08091E8008B778093E8009115C0
:105A900009F493CDE090F002F090F102E981E11475
:105AA000F10409F496C0EE3F09F0B6C08A81833054
:105AB00020F08550833008F0AFC0EA81EE3008F066
:105AC000ABC0F0E0E955FA4C27C680E090E075CE17
:105AD0000E94F62310926E0510926D050E94ED094A
:105AE00098CE44EFE42EFF24F3945DE8C52E59E0F0
:105AF000D52E823209F4B1CE833209F43CC085310F
:105B000009F0A3CEF0E0EB50F94FE491EE2EF12C2A
:105B100075E4C72E79E0D72EA0CEF0E0EF5FF84F06
:105B2000E491EE2EF12CB2EBCB2EB8E0DB2E95CE2D
:105B3000F0E0E250F94FE491EE2EF12CA3EACA2EE8
:105B4000A8E0DA2E8ACEE695F0E0E550F94FE49130
:105B5000EE2EF12CF5ECCF2EF8E0DF2E7ECEE69582
:105B6000F0E0E850F94FE491EE2EF12CEBEECE2E62
:105B7000E8E0DE2E72CE8E2F63E08ED5E92FF0E0C6
:105B8000EE50F94FE491EE2EF12C64EDC62E67E154
:105B9000D62E63CE30E2C32ED12C9E012F5F3F4F15
:105BA00079018091E80085FD0AC08091E8008B773B
:105BB0008093E8000E94810D811599F362CF809156
:105BC000F100D7018D937D01B1E0CB1AD10849F7DF
:105BD00058CFE43148F4E11551F0E150E33138F4A5
:105BE000F0E0EB54FA4C98C5EE3F09F466CF8FEF26
:105BF000898312C01A8289E08B830EC08A81823029
:105C000081F08330B1F0813091F70E94BC0C8AD5CD
:105C10006B837C838D839E83CE0101960E94D10D80
:105C2000CCCC88E290E081D61B821C821D828E83C0
:105C3000F3CF8091EB029091EC02892B69F3FE0186
:105C40003196D8018C9111969C910E5F1F4F9283D3
:105C500083833296B2E00B3E1B0799F7DDCF8A8132
:105C6000823029F66B817C818D819E815BD588E2B3
:105C700090E07CD6D1CF4C816B818A810E944F14F9
:105C80009827892798279E838D83C6CF2D813E81B3
:105C90003227232732274C816B818A810E94500F43
:105CA000BBCF0E94F515B8CF8A81823891F1B0F44C
:105CB0008038E9F0813809F0AFCF60E08B810E9435
:105CC00052199B818091AF0491111AC08E7F8093ED
:105CD000AF041092AE040E9462089ECF833809F090
:105CE0009BCF20E04091B2046C818B8106C020E004
:105CF0004B816091B1048091B0040E94A5188CCFB3
:105D000081608093AF0460E0869586950E94521969
:105D100083CF8B818093B3047FCF8A818238E1F077
:105D200060F48038A1F0813809F076CF8091AF041B
:105D300080FF10C0869586955FCF833809F06CCFC1
:105D40008091B0048B838091B1048C8365CF809166
:105D5000B20452CF80E050CF8091B3044DCF0E9467
:105D600054088FEA94E00E94651856CF80E18A8338
:105D700053CF1A828FE840CF8C818D3108F04CCF01
:105D80008A809B80982489249824A12CB12C8E0190
:105D90000F5F1F4F7801E80EF11CE016F10609F4C1
:105DA0003BCF80E0EFE88E169104A104B10420F40B
:105DB000C4018F589C4FB9D5D80114968C930F5FAE
:105DC0001F4FBFEF8B1A9B0AAB0ABB0AE6CF80912D
:105DD000EB029091EC02892B09F41ECF8C818D315E
:105DE00008F01ACF882E912CA12CB12CCA80DB8010
:105DF000DC24CD24DC24E12CF12C8E010F5F1F4F1D
:105E0000412C512C3201481459046A047B0408F0D7
:105E100003CFEFE8CE16D104E104F10438F4D80141
:105E200014966C91C6018F589C4FA0D5BFEF4B1AAA
:105E30005B0A6B0A7B0AEFEFCE1ADE0AEE0AFE0A55
:105E40000F5F1F4FE0CF55D9E7CE84E090CF8C8114
:105E50008D3108F0E1CE882E912CA12CB12CCA8076
:105E6000DB80DC24CD24DC24E12CF12C412C512CD2
:105E700032018E010B5F1F4F481459046A047B04E2
:105E800008F0CACE80E0F8E5CF16F2E0DF06E104C4
:105E9000F10418F4C601899648D5D8018D938D0177
:105EA000BFEF4B1A5B0A6B0A7B0AEFEFCE1ADE0AD2
:105EB000EE0AFE0AE1CF2C81022F10E02D3108F00E
:105EC000ABCE8A819B819827892798272C01612C4A
:105ED000712C8835F2E09F0708F09ECE822E912C1F
:105EE000A12CB12C48E552E060E070E0441955095E
:105EF00066097709421751056105710508F48CCED2
:105F00002091EB023091EC02232B09F03EC01C01E2
:105F100029E2220E311C80FBEE24FF24E0F880FFF2
:105F20000BC0889602D59D818927982789278115DE
:105F30009C4711F48FEF8D83D501C401840D951D0D
:105F4000A61DB71D80FF19C0680141E0C41AD10821
:105F5000CE0105968C0D9D1D9CA78BA7C101800FBE
:105F6000911FE3D4ABA5BCA59C9181159C4721F45E
:105F70008FEFEBA5FCA580838601FE013196EE0D27
:105F8000FF1D2FEFE016F10638F08E010F5F1F4F57
:105F9000C12CD12C760125C09481858181159C4727
:105FA00011F42483258342E0E40EF11C3296EACFFB
:105FB00088E5481682E058066104710430F4D8017F
:105FC00014966C91C2018996D1D4BFEFCB1ADB0A2B
:105FD000EB0AFB0AEFEF4E1A5E0A6E0A7E0A0F5FAB
:105FE0001F4FC814D904EA04FB0410F315CE8091A6
:105FF000EB029091EC02892B09F40ECECE010196B2
:106000000E94D10DFFEF21EE34E0F15020403040EE
:10601000E1F700C00000A1CA88E0E3E2F1E0DE01A0
:10602000919601900D928A95E1F7FE0132968FE1EB
:10603000DF011D928A95E9F786E0898388E07F96E3
:10604000DE01159601900D928A95E1F7E5CD8CEC75
:10605000898381E08A831B821C82DECD8B819C81B7
:10606000092E000CAA0BBB0B25E0880F991FAA1F55
:10607000BB1F2A95D1F7AC01BD01405E5F4F6F4F4A
:106080007F4F481759076A077B0708F4C5CD8C3C3A
:10609000E1E09E07A105B10508F0BECD4D3CF1E061
:1060A0005F076105710520F04CEC51E060E070E0A5
:1060B000481B590BBC016B5F784FCE010196FBD397
:1060C000ABCD4AE150E06FEF70E0CE01079616D4F9
:1060D0008091EB028983EA821B821C8282E08D839D
:1060E0008BE0A5CD81E090E09093F1028093F002E7
:1060F00082E390E09093E0028093DF020E94650BC0
:106100009093DE028093DD0287CDE114F10481F1EA
:10611000D090E102C090E6020091DD021091DE0213
:106120000E94650B801B910B8536910540F1C3FEE3
:1061300026C0D0FE24C00E94650B9093DE0280939F
:10614000DD028091DF029091E00201979093E002DE
:106150008093DF02892B61F41092F1021092F00219
:1061600081E090E09093EC028093EB02E12CF12C23
:106170008091EB028983EA828091DF023DCD82E348
:1061800090E09093E0028093DF02F2CF1092EC0255
:106190001092EB0241CD40E250E06FEF70E0CE0193
:1061A0000196ACD339CDEB81E73008F035CDF0E086
:1061B000E853FA4CB1C2FE0134968DE1DF011D9225
:1061C0008A95E9F788E089838A8316CD8C819AE0E5
:1061D000F92E8E010F5D1F4FF8012F2D11922A9578
:1061E000E9F7B8010E9444178983F801DE0112968D
:1061F00001900D92FA94E1F70FCD1C818AE0FE0127
:106200003596DE01919601900D928A95E1F789A16C
:106210009AA10E94BB099AA389A38BA19CA10E9469
:10622000BB099CA38BA38DA19EA10E94BB099EA329
:106230008DA38FA198A50E94BB0998A78FA38FEF6C
:10624000183060F43AE0139FB00111246F577D4F6E
:106250004AE050E0CE018196A7D380E089830E9476
:10626000C809DACC2C816AE0CE018196DC01E62FE8
:106270001D92EA95E9F7283008F044C0629FB0010A
:1062800011246F527D4F4AE050E03FD380E0898374
:106290008AE0FE01B196DE011296D4CE1C818AE01E
:1062A000FE013596DE01919601900D928A95E1F7F7
:1062B00089A59AA50E94BB099AA789A78FEF1830D4
:1062C00060F4FAE01F9FB00111246F527D4F4AE045
:1062D00050E0CE01819668D380E089830E948116C8
:1062E0009BCC2C816AE0CE018196DC01E62F1D92C9
:1062F000EA95E9F7283030F4629FB00111246F5D10
:106300007C4FC1CF8FEFC3CF1C818AE0FE01359651
:10631000DE01919601900D928A95E1F78BA19CA1E7
:106320000E94BB099CA38BA38FEF183060F4FAE0A6
:106330001F9FB00111246F5D7C4F4AE050E0CE01F9
:10634000819632D380E089830E94C51665CC2B30BC
:10635000310508F020CB4DCB2B30310508F0D5CAE4
:1063600002CB8091BE02811509F4B7C9B0E1B9BD75
:10637000E2E1E9BD09B400FEFDCF8091D8008F7D38
:106380008093D8008091E00082608093E00080914B
:10639000E00081FDFCCF0E94AC109FC91F921FB688
:1063A0001F9211248F939F93AF93BF938091BD024F
:1063B000811113C08091260290912702A09128029A
:1063C000B09129024196A11DB11D809326029093A0
:1063D0002702A0932802B0932902BF91AF919F9109
:1063E0008F911F901FBE1F90189578941F921FB613
:1063F0001F9211248F939F93AF93BF938091260296
:1064000090912702A0912802B09129020196A11D26
:10641000B11D8093260290932702A0932802B09387
:106420002902BF91AF919F918F911F901FBE1F9026
:1064300018951F920F920FB60F9211242F933F932E
:106440004F935F936F937F938F939F93AF93BF937C
:10645000EF93FF938091E10082FF09C08091E200F9
:1064600082FF05C08091E1008B7F8093E1008091E5
:10647000DA0080FF24C08091D80080FF20C0809186
:10648000DA008E7F8093DA008091D90080FFA9C066
:1064900080E189BD82E189BD09B400FEFDCF81E0C4
:1064A0008093ED0280911502811109C00E94B20D06
:1064B0000E940F0E8091E20084608093E200809140
:1064C000E10080FF1AC08091E20080FF16C0809139
:1064D000E2008E7F8093E2008091E20080618093F1
:1064E000E2008091D80080628093D80019BC85E0DA
:1064F0008093ED0283E0809320018091E10084FF8E
:106500002FC08091E20084FF2BC080E189BD82E131
:1065100089BD09B400FEFDCF8091D8008F7D8093A6
:10652000D8008091E1008F7E8093E1008091E200AD
:106530008F7E8093E2008091E20081608093E20090
:1065400080911402811509F452C084E08093ED0219
:106550008091ED02843009F052C082E080932001E6
:106560008091E10083FF2CC08091E20083FF28C06E
:106570008091E100877F8093E10082E08093ED02CB
:10658000109214028091E1008E7F8093E10080914F
:10659000E2008E7F8093E2008091E2008061809330
:1065A000E20042E060E080E00E94DF0D8091F000B8
:1065B00088608093F00081E08093200180931F0128
:1065C000FF91EF91BF91AF919F918F917F916F91CB
:1065D0005F914F913F912F910F900FBE0F901F90A1
:1065E000189519BC1092ED021092150268CF809197
:1065F000E30087FF02C083E0A9CF81E0A7CF81E05D
:10660000ADCF1F920F920FB60F921124EF92FF920F
:106610000F931F932F933F934F935F936F937F93AA
:106620008F939F93AF93BF93CF93EF93FF9309EE15
:1066300010E0F8018081C091EC008F70C795CC27E5
:10664000C795C82B108280EFE82EF12CF7018081CE
:10665000877F808378940E94ED10F8011082F70103
:10666000808188608083CF70F801C083FF91EF91B3
:10667000CF91BF91AF919F918F917F916F915F91DA
:106680004F913F912F911F910F91FF90EF900F909D
:106690000FBE0F901F901895992778E0880F991FCB
:1066A000961708F0961B881F7A95C9F7809508956C
:1066B00087FB082E062687FD819567FD6195ECDF37
:1066C0000EF4919507FC81950895AA1BBB1B51E11F
:1066D00007C0AA1FBB1FA617B70710F0A61BB70B52
:1066E000881F991F5A95A9F780959095BC01CD01F7
:1066F000089597FB072E16F4009406D077FD08D076
:10670000E4DF07FC05D03EF4909581959F4F0895F6
:10671000709561957F4F0895EE0FFF1F0590F491DE
:10672000E02D0994692796276927782787277827F6
:1067300008952F923F924F925F926F927F928F9225
:106740009F92AF92BF92CF92DF92EF92FF920F9300
:106750001F93CF93DF93CDB7DEB7CA1BDB0B0FB60A
:10676000F894DEBF0FBECDBF09942A8839884888C7
:106770005F846E847D848C849B84AA84B984C8845D
:10678000DF80EE80FD800C811B81AA81B981CE0F54
:10679000D11D0FB6F894DEBF0FBECDBFED01089539
:1067A000002E083090F0982F872F762F652F542FCA
:1067B000432F322F22270850F4CF220F331F441FBC
:1067C000551F661F771F881F991F0A95B2F7002D66
:1067D000089597FD1094002E083098F00850232F4C
:1067E000342F452F562F672F782F892F912DF4CFD7
:1067F000159497958795779567955795479537950C
:1068000027950A95AAF71124002D08958F929F923B
:10681000AF92BF92CF92DF92EF92FF92CF93DF932E
:10682000EC01688179818A819B81611571058105FF
:10683000910521F464E279ED8BE597E02DE133EFEA
:1068400041E050E0C8D049015A019B01AC01A7EAE0
:10685000B1E4DDD06B017C01ACEEB4EFA501940195
:10686000E2D0DC01CB018C0D9D1DAE1DBF1DB7FF1D
:1068700003C00197A109B04888839983AA83BB8389
:106880009F77DF91CF91FF90EF90DF90CF90BF90F7
:10689000AF909F908F900895B9CF80E091E0B6CFF0
:1068A000A0E0B0E08093000190930101A093020169
:1068B000B09303010895FB01DC0102C005900D9225
:1068C00041505040D8F70895FC014150504030F0FD
:1068D00001900616D1F73197CF010895882799279F
:1068E0000895FB01DC0104C08D910190801921F411
:1068F00041505040C8F7881B990B0895DC0101C036
:106900006D9341505040E0F70895DC01CB01FC014C
:10691000F999FECF06C0F2BDE1BDF89A319600B4F8
:106920000D9241505040B8F70895F999FECF92BDAD
:1069300081BDF89A992780B50895A6E1B0E044E0BA
:1069400050E0E5CFA8E1B0E042E050E0E0CFDC016C
:10695000A40FB51F4150504040F0CB01840F951F4C
:106960002E9105D041505040D8F70895262FF9991F
:10697000FECF92BD81BDF89A019700B4021639F09E
:106980001FBA20BD0FB6F894FA9AF99A0FBE08956F
:106990000396272FECDFEADF252FE9DF242FE7CF4F
:1069A0000196272FE4DFE2CFDC01CB0102C02D915D
:1069B00005D041505040D8F70895262FF999FECFC1
:1069C0001FBA92BD81BD20BD0FB6F894FA9AF99A0C
:1069D0000FBE01960895052E97FB16F400940FD074
:1069E00057FD05D024D007FC02D046F408C05095CE
:1069F0004095309521953F4F4F4F5F4F08959095AB
:106A00008095709561957F4F8F4F9F4F089531D03E
:106A1000A59F900DB49F900DA49F800D911D1124F2
:106A20000895B7FFF4CFF3DF821B930B0895A1E223
:106A30001A2EAA1BBB1BFD010DC0AA1FBB1FEE1FF8
:106A4000FF1FA217B307E407F50720F0A21BB30B43
:106A5000E40BF50B661F771F881F991F1A9469F7BF
:106A600060957095809590959B01AC01BD01CF011B
:106A70000895A29FB001B39FC001A39F700D811D17
:106A80001124911DB29F700D811D1124911D089537
:106A9000F894FFCF0D0C120C140C190C290C290CB6
:106AA000290C290C290C290C290C290C1B0C1F0C56
:106AB000220C270C370C3D0C410CCA11F011F611B9
:106AC000F011F61148126912F6116F137C13C71DED
:106AD0002F1ECF1D991D9D1DD31DA11DD71DE31D6B
:106AE000AD1D281EB11DE71DB51DEB1D101EB91DE6
:106AF000EF1D171EBF1DF51DFD1DA51DDB1DA91DCD
:106B0000DF1DC31DF91D071E201E261E931DCB1D54
:106B1000361E651D6B1D581D5F1D711D771D7D1D6A
:106B2000561E6D1E711E751E791E7D1E811E851ED0
:106B3000891E8D1E911E5E1F5E1F971F971F492085
:106B40006420BD1FBD1F6920DC20ED20ED200C302E
:106B500027302E300C2E0C2E613072308530C6302E
:106B6000CB300C2E0C2E0C2ED330FA2DFE2D2F2ECA
:106B70003B2E462E512E542E8D2EAF2EF72DF72F55
:106B8000B62EB92EBC2EE72E232F252F272F5B2FB5
:0E6B9000DB30E630FD3032314E317131843170
:106B9E000100000001020118191A1B1C1D1E1F20E6
:106BAE0021620B140F2A0F2F0F340F0B0F00000151
:106BBE00000101097A78FE4FB4CBE4004422B6847A
:106BCE00016201AC008A02A302C3020001020202AA
:106BDE00020606060909090909090F0F0F0F0F0F03
:106BEE001515151818181818181818181822232300
:106BFE0023232323F1F0C6F5F4F6F7676636353412
:106C0E009796949593379192E200E900EA00B500C9
:106C1E00B600B700CD008301CC008A019201940129
:106C2E002102230224022502260227022A02B30091
:106C3E00B4006F0070009F01CB019F02A002E20022
:106C4E00E900EA00B500B600B700CD008301CC0024
:106C5E008A019201940121022302240225022602B6
:106C6E0027022A02B300B4006F0070009F01CB010F
:046C7E009F02A002CF
:00000001FF
